:0200000480007A
:10000000B72F0000938F0F8073900F3015A8130047
:100010000000130000001300000013000000130094
:100020000000130000001300000013000000130084
:100030000000130000001300000013000000010086
:10004000970200009382020C73905230814001416C
:100050008141014281420143814301448144014580
:100060008145014681460147814701488148014950
:100070008149014A814A014B814B014C814C014D20
:10008000814D014E814E014F814F971102009381A6
:1000900021D3170502001305E55697A503009385A4
:1000A000E580014611221705020013052548970532
:1000B00002009385A5500146C52817A50300130526
:1000C000257F97B503009385657E37B6ABAB1306E6
:1000D000B6BAD92817B103001301817DEF60B020B3
:1000E000860293D21200F512638802008242110147
:1000F0006F00001073002030824211017300203025
:10010000711116C0F3222034E3CC02FC82421101AB
:10011000130141F806C20AC40EC612C816CA1ACC88
:100120001ECE22D026D22AD42ED632D836DA3ADCC7
:100130003EDEC2C0C6C2CAC4CEC6D2C8D6CADACC97
:10014000DECEE2D0E6D2EAD4EED6F2D8F6DAFADCA7
:10015000FEDE73252034F32510340A8601A07310C7
:10016000153492402241B2414242D2426243F243AC
:10017000025492542255B2554256D2566257F25703
:10018000064896482649B649464AD64A664BF64B33
:10019000065C965C265DB65D465ED65E665FF65F83
:1001A0001301C1077300203010C16374B50011053D
:1001B000E5BF828000000000000000000000000099
:1001C000000000000000000000000000000000002F
:1001D000000000000000000000000000000000001F
:1001E000000000000000000000000000000000000F
:1001F000197106C00AC20EC412C616C81ACA1ECC8D
:1002000022CE26D02AD22ED432D636D83ADA3EDCC6
:1002100042DEC6C0CAC2CEC4D2C6D6C8DACADECC96
:10022000E2CEE6D0EAD2EED4F2D6F6D8FADAFEDCA6
:100230009702020083A2C23223A02200F3221034CC
:1002400096DEEF00002B170102000321613102410D
:10025000F65273901234B72200009382028873A082
:10026000023082403242C2425243E24372448254DC
:100270001255A2553256C2565257E2577258864806
:100280001649A649364AC64A564BE64B764C865C1A
:10029000165DA65D365EC65E565FE65F0961730059
:1002A0002030970202009382E23523A0120023A29D
:1002B000220023A4320023A6420023A8520023AA2E
:1002C000620023AC720023AE820023A0920223A21C
:1002D000A20223A4B20223A6C20223A8D20223AA06
:1002E000E20223ACF20223AE020323A0120523A2F2
:1002F000220523A4320523A6420523A8520523AADA
:10030000620523AC720523AE820523A0920723A2C7
:10031000A20723A4B20723A6C20723A8D20723AAB1
:10032000E20723ACF207EF4030531701020003212C
:1003300021230241F65273901234B72200009382B7
:10034000028873A0023082403242C2425243E243EA
:10035000724482541255A2553256C2565257E25731
:10036000725886481649A649364AC64A564BE64B45
:10037000764C865C165DA65D365EC65E565FE65FB1
:10038000096173002030970202009382A22783A0A4
:10039000020003A1420083A1820003A2C20083A243
:1003A000020103A3420183A3820103A4C20183A427
:1003B000020203A5420283A5820203A6C20283A60B
:1003C000020303A7420383A7820303A8C20383A8EF
:1003D000020403A9420483A9820403AAC20483AAD3
:1003E000020503AB420583AB820503ACC20583ACB7
:1003F000020603AD420683AD820603AEC20683AE9B
:10040000020703AFC20983AF820782807370043092
:10041000197106C00AC20EC412C616C81ACA1ECC6A
:1004200022CE26D02AD22ED432D636D83ADA3EDCA4
:1004300042DEC6C0CAC2CEC4D2C6D6C8DACADECC74
:10044000E2CEE6D0EAD2EED4F2D6F6D8FADAFEDC84
:100450009702020083A2C21023A0220086DEEF20B2
:10046000205A170102000321A10F0241F652739096
:100470001234B72200009382028873A002308240B7
:100480003242C2425243E243724482541255A25550
:100490003256C2565257E257725886481649A649F4
:1004A000364AC64A564BE64B764C865C165DA65DD0
:1004B000365EC65E565FE65F09617300203073707A
:1004C000043001A07310453082807325403073F0F2
:1004D00043308280970700009387A7FE232EB5FE46
:1004E0002322C5FA232635F82320F5F8130505F84D
:1004F0008280411106C6EF405033EF10503601E5BF
:10050000B24041018280B24041016F20604F9307A9
:1005100085007D575CC118C55CC51CC9232005003A
:1005200082802328050082805C41DCC1984798C501
:1005300098474CC38CC788C91C4185071CC1828061
:100540009041FD57130785006314F60039A83E87D4
:100550005C439443E37DD6FEDCC18CC798C54CC395
:1005600088C91C4185071CC1828018495C43EDB7CE
:10057000584114451C4914C71845544154C3D84325
:100580006314A7001845D8C32328050088437D15A8
:1005900088C38280411122C406C626C23C412A84F7
:1005A00081EF1C41A5CF01451C5C85071CDCB240D6
:1005B0002244924441018280B2841DE608453E8671
:1005C000EF30304B1C4434405840B6971CC4E3EC29
:1005D000E7FC1C4001451CC41C5C85071CDCB240C8
:1005E000224492444101828048453E86EF30704863
:1005F00038405C4414403307E040BA975CC463F56C
:10060000D7005C403E9758C48947E39EF4F81C5CD1
:10061000D9DB1C5C0145FD171CDC79B74841EF2094
:10062000302F2322040049B7011106CE22CC26CA5E
:1006300060492AC615C0185C5C5C6365F70073707E
:10064000043001A0185C8144636BF700F2406244FF
:100650002685D244056182807370043001A02E8605
:1006600022856C00053F3844FD57AA846306F700D5
:100670003C4485073CC4D9BF5C50E9DB1305440208
:10068000EF20207A61D58544D1B73041AE8701CEC5
:100690004C455841B2954CC563E4E5000C414CC54E
:1006A0003E856F30103D8280797122D406D62A842F
:1006B00026D24AD04ECE52CC56CAEF20102E3C4401
:1006C000635CF002130A4402FD590549644889C875
:1006D000985CDC5C22C66367F7067370043001A087
:1006E0005C5099CB5285EF20C0732DED3C44FD1733
:1006F0003CC43C44E34CF0FCFD573CC4EF20302CA0
:10070000EF20B0297C406352F0021C4899CF93043B
:1007100004012685EF20E07029E97C40FD177CC0AC
:100720007C406354F0001C48EDF7FD577CC0EF207F
:100730001029B250225492540259F249624AD24AC4
:1007400045618280985CE373F7FA01466C00268568
:100750009135BC44AA8A638D3701BC448507BCC46B
:10076000E3962AF9EF20300C51B7EF20D00B75B784
:10077000DC50FDD713854402EF20A06A75D1DDB7A8
:1007800029CD011122CC2A8406CE26CA4AC84EC6DB
:100790002E89EF20902024404C5C8329040026857C
:1007A000EF6000167D57232C0402B3079540CE97C7
:1007B0004E9578C048C0232434015CC438C463110A
:1007C00009021C488DE7EF20901FF2406244D2449A
:1007D0004249B2490545056182807370043001A029
:1007E000130504012D33130544021533E9BF130526
:1007F0000401EF2000638547E317F5FC0139E1B7F9
:1008000001E57370043001A0011126CA4AC84EC622
:1008100006CE22CCAA842E89B289B5C9EF60400EDB
:1008200013059505EF30B00C2A8425C9930785057B
:100830001CC144DC23202405EF20301624404C5CEE
:10084000032904002685EF60A00BFD56232C04022B
:10085000B30795403307A900CA9774C058C05CC459
:1008600034C4130504012324240155311305440223
:100870007939EF20D01423083405232A0404228573
:10088000F2406244D2444249B24905618280130574
:100890008005EF30D0052A8401E57370043001A093
:1008A00000C041BF797126D2AA841305800522D4E5
:1008B00006D64AD04ECE52CCEF3070032A8421C9DE
:1008C000232C0502FD577CC10547130A05013CC4D2
:1008D000528558DC23220400232004002324040032
:1008E000232604002320040423089404232A040458
:1008F0003939130944024A8519393C4002C28DC373
:100900007370043001A022854533EF101011228549
:10091000B250225492540259F249624A456182808F
:10092000EF20E07201E59247639C070AEF20F00692
:10093000185C5C5C8144FD596362F7069247C1C351
:1009400081E42800EF200061EF207007EF10E067DE
:10095000EF20B0047C4063943701232204043C441C
:100960006394370123240404EF2070054C00280011
:10097000EF20606049F9EF205002185C5C5C630373
:10098000F704EF20D00322850533EF1010098544CA
:10099000EF20B000185C5C5CE372F7FA304021E6AF
:1009A0001C40ADC701451C5C784885071CDC39CB71
:1009B00081452285953985476313F500813CEF20F9
:1009C0001000B1B7EF20A07F92455285EF2020277D
:1009D0002285D939EF1070045DF90D3C85444DBF77
:1009E0007370043001A008448145EF3090081C4426
:1009F00034405840B6971CC4E3E6E7FA1C40014572
:100A00001CC455B75C5089EB5DD94DBF4840EF2001
:100A100020702322040041BF4A85EF208040854793
:100A2000E31FF5F861BF01E57370043001A0637541
:100A3000B5007370043001A0411122C409462E8410
:100A4000814506C6753B11C500DDB2402244410117
:100A500082807370043001A0397106DE22DC26DA50
:100A60004AD84ED652D456D25AD032C66300051058
:100A70006388050E89476399F600585D85476305CD
:100A8000F7007370043001A0B6842E892A84EF2009
:100A9000005C11E5B24781C77370043001A0EF20FC
:100AA000C06F185C5C5C8149094B7D5A930A040154
:100AB0006367F706638F640BB24763890712639518
:100AC00009002808EF200049EF20606FEF10E04F89
:100AD000EF20A06C7C4063944701232204043C4433
:100AE0006394470123240404EF20606D6C00280800
:100AF000EF2060486316050EEF20206A185C5C5CEE
:100B00006302F704EF20A06B2285793EEF10E070BE
:100B10008549EF208068185C5C5CE37DF7F8304025
:100B200039CA6399040C0844CA85EF3080741C44A8
:100B300034405840B6971CC463E1E7041C400145AB
:100B40001CC42DA8EF20A067B2455685EF20200FCA
:100B50002285993EEF10606C45FD4D38854955BFA3
:100B60003C41E38907F07370043001A073700430D6
:100B700001A0304005EE1C40D5C301451C5C7848FF
:100B800085071CDC51C7A6852285793C854763040F
:100B9000F508EF20C0620545F2506254D254425924
:100BA000B259225A925A025B216182804844CA8516
:100BB000EF30206C3C4058441440B307F0403E975F
:100BC00058C46378D7005840BA975CC48947E39605
:100BD000F4FA1C5CDDD31C5C0145FD171CDC79BFFD
:100BE0002285D934EF10606301457DB7EF20205D89
:100BF00001455DB74844CA85EF30A0673C40584482
:100C00001440B307F0403E9758C4E371D7FC65BF6A
:100C10005C5099EB3DDDEFF06FFFA5BF4840EF2042
:100C2000204F2322040099BF13054402EF20601FC8
:100C30008547E310F5F6C5B70DC5411122C426C29C
:100C400006C64AC0032945002A84EF20803F81441C
:100C5000630CA900B2402244268502499244410116
:100C600082807370043001A05C448544FD175CC42D
:100C7000F5F38146014681452285F93BE1BF39CD37
:100C8000A9C9011122CC26CA4AC852C406CE4EC6F2
:100C90008947B68432892E8A2A846399F600585D82
:100CA00085476300F7067370043001A03938185C7B
:100CB0005C5CAA896367F70281444E85EFF09F80F0
:100CC000F240624426854249D244B249224A056133
:100CD00082803C41DDD77370043001A07370043012
:100CE00001A0304049E21C40DDCB1C5C7D578507EC
:100CF0001CDC3C446388E7083C44854485073CC4CD
:100D00006DBFEFF08FFC185C5C5CAA89636DF70225
:100D1000304071DA4844D285EF30A0553C40584409
:100D20001440B307F0403E9758C46375D70058404D
:100D3000BA975CC48947E39AF4FA1C5CDDD71C5C63
:100D4000FD171CDC5DB7304059DE4844D285EF30DA
:100D500040523C4058441440B307F0403E9758C4BA
:100D6000E367D7FCD9BFDDF40844D285EF3060508B
:100D70001C4434405840B6971CC4E3E8E7F61C40D6
:100D80001CC4A5B77C4895C3A685228571388544C7
:100D9000E31595F2E30309F22320990039BF484097
:100DA000EF2000372322040089B75C508544E38696
:100DB00007F013054402EF20C00669FDFDBD31CDEB
:100DC0003C4181C77370043001A01C41B1CB0111BB
:100DD00022CC26CA2A844AC84EC606CE2E89EFF0F7
:100DE000CFEE185C5C5CAA898144637DF7001C5CD3
:100DF0007D5785071CDC3C446389E7023C448544FD
:100E000085073CC44E85EFF0EFEBF2406244268547
:100E10004249D244B249056182807370043001A016
:100E20005C41D5D77370043001A07C4891CB8145DB
:100E30002285EFF06FFF8547630BF5008544D9B736
:100E40005C50EDDF13054402EF10B07D65D9E30778
:100E500009FE85472320F900D5B7397106DE22DC6B
:100E600026DA4AD84ED652D432C6630A050E6382B9
:100E7000050EB6892E892A84EF20601D11E5B24740
:100E800081C77370043001A0EF2020311C5CD1E7D2
:100E9000B247638E07102808EF20C00BFD54130AD9
:100EA000440239A8EF20A0312285EFF0EFFFEF10C8
:100EB000C036EF20802E1C5CADE3B2476389070E7D
:100EC000EF20E02FEF106010EF20202D7C40639486
:100ED0009700232204043C446394970023240404D1
:100EE000EF20E02D6C002808EF20E00855E9EF2006
:100EF000C02A1C5CC5FBEF20802C1C40BDC7B2453E
:100F00005285EF10D0532285EFF00FFAEF10E0304A
:100F100031C9EF2080281C5CCDD3CA85228544448A
:100F2000EFF0AFF6639B09041C5C1840FD171CDC56
:100F300001E7EF20402D48C01C48B9EBEF202028E6
:100F40000545F2506254D2544259B259225A216195
:100F500082803C41E38F07F07370043001A073700E
:100F6000043001A0EFF08FCA6DB7EF200023484096
:100F7000EF20E00FEF20A02459B75C5044C4DDDF20
:100F800013054402EF10F06955D9EFF02FC87DB773
:100F900013050401EF10F0688547E311F5FAF5B782
:100FA0002285EFF06FF0EF104027014559BFEF2089
:100FB0000021014579B71DC9411122C44AC006C6A6
:100FC00026C244412E892A84EF20A0076383A4020D
:100FD00081464A8681452285493585476300F50269
:100FE000B24022449244024941018280737004302D
:100FF00001A05C44054585075CC4DDB75C448507FA
:101000005CC4F9BF15CDADC9011122CC26CA4AC8AE
:101010004EC652C42A8406CE3289AE89EFF0EFCA9A
:101020001C5C2A8A814485E35285EFF0AFC9F24007
:10103000624426854249D244B249224A05618280EF
:101040007370043001A0304001CE4C445C40B29536
:101050004CC463E4F5000C404CC44E85EF30602175
:101060001C5C7D57FD171CDC7C40638CE7007C40DA
:10107000854485077CC04DBF3C41D9D7737004308F
:1010800001A01C4899E3854445B713050401EF10FE
:10109000505975D9E30909FE85472320F900E5B7C2
:1010A00021C93C41A1CDA1CB011122CC26CA4AC8FD
:1010B00052C42A8406CE4EC62E8AEFF00FC11C5CA5
:1010C0002A89814491CB8329C400D2852285EFF0FF
:1010D000CFDB8544232634014A85EFF0AFBEF240D2
:1010E000624426854249D244B249224A056182803F
:1010F0007370043001A07370043001A0EDDF7370D1
:10110000043001A001E57370043001A0411122C434
:101110002A8406C6EF206008005CEF20400AB24037
:10112000228522444101828001E57370043001A0D0
:10113000411106C622C42A84EF2020061C5C405CB4
:101140001D8CEF20C0072285B240224441018280DD
:1011500019C1085D82807370043001A01DCD97878E
:10116000030093876770D843630CE502D847630C8C
:10117000E504D84B6307E504D84F6302E504D85370
:10118000630DE502D8576308E502D85B6303E50207
:10119000D85F630EE5006F30A0077370043001A0C4
:1011A00001470E07BA9723A007006F3060061D475E
:1011B000CDBF1947FDB71547EDB71147DDB70D474F
:1011C000CDB70947F9BF0547E9BF684582806CC5BF
:1011D000828003450505828009C5085D1335150029
:1011E00082807370043001A019C51C5D485D1D8D9F
:1011F0001335150082807370043001A097870300B7
:1012000093878766984305C3984705C7984B05C7DA
:10121000984F05C7985305C7985705C7985B15C7DA
:10122000985F15C3828001470E07BA978CC3C8C365
:1012300082800547D5BF0947C5BF0D47F5B71147A0
:10124000E5B71547D5B71D47C5B71947F1BF97870C
:10125000030093876761D8436308E502D847630BAF
:10126000E502D84B630AE502D84F6309E502D8537B
:101270006308E502D8576307E502D85B6308E50217
:10128000D85F6303A702828001470E07BA9723A0A5
:10129000070082800547D5BF0947C5BF0D47F5B791
:1012A0001147E5B71547D5B71D47C5B71947F1BF72
:1012B000797122D426D24AD02A8406D64ECE52CC78
:1012C00056CAAE843289EF10506D7840FD576314D2
:1012D000F700232204043844FD576314F700232445
:1012E0000404EF10D06D1C5C99E74A86A6851305AF
:1012F0004402EF10D027EF10506A3C44635CF002C8
:10130000130A4402FD590549644889C8985CDC5CAD
:1013100022C66367F7067370043001A05C5099CB56
:101320005285EF10103035ED3C44FD173CC43C4471
:10133000E34CF0FCFD573CC4EF107068EF10F06513
:101340007C406352F0021C4899CF93040401268527
:10135000EF10302D31E97C40FD177CC07C40635498
:10136000F0001C48EDF7FD577CC0EF105065B250FF
:10137000225492540259F249624AD24A456182800B
:10138000985CE373F7FA01466C002685EFF08FA0B6
:10139000BC44AA8A638D3701BC448507BCC4E3956D
:1013A0002AF9EF10504849B7EF10F0476DB7DC50FD
:1013B000FDD713854402EF10D02675D1DDB701E5C6
:1013C0007370043001A0411126C2AA840A051305D6
:1013D000950522C406C64AC0EF2070512A843DC13B
:1013E000930785051CC191473CC144DDEF10F05ABD
:1013F00024404C5C032904002685EF506050FD56C4
:10140000232C0402B30795403307A900CA9774C080
:1014100058C05CC434C41305040123242401EFF034
:101420000F8F13054402EFF08F8EEF1050592308F1
:101430000404232A04042285B2402244924402492F
:10144000410182807370043001A0411122C426C280
:101450004AC02A8406C62E89EF1030547C48814445
:1014600091CBEF10D055B2402244268502499244D8
:10147000410182801C5C8144EDF7232A24058544C8
:10148000CDB77C496385B70081473E858280185D72
:10149000814765FF411122C42A8406C6EF10F04F30
:1014A000232A0404EF10B051B240224485473E8500
:1014B0004101828001112E8681466C0006CE02C653
:1014C000693AF240324505618280011106CE22CC94
:1014D00026CA02C605C12A84EFE03FFF1C5CAA842D
:1014E00089EF2685EFE01FFEF24062443245D24488
:1014F000056182807370043001A0304001CE4C44FD
:101500005C40B2954CC463E4F5000C404CC46800E8
:10151000EF2030561C5C7D57FD171CDC7C40638639
:10152000E7007C4085077CC06DBF1C48DDDB1305F0
:101530000401EF10100F75B71DC179714ECE52CC5A
:1015400006D63E8A22D426D24AD056CA5AC85EC689
:10155000A547BA8963F8E7007370043001A073707F
:10156000043001A02A8BAE843289B68BC28A63070D
:10157000082213050006EF2090372A84630B05200C
:101580000A09232855034A869305500A5685EF20F9
:10159000505C03C704001C587119230AE40203C7F6
:1015A00004003E991379C9FF79C783C71400A30AC1
:1015B000F40283C71400E1C383C72400230BF402A1
:1015C00083C72400CDCB83C73400A30BF40283C7A9
:1015D0003400D5C383C74400230CF40283C74400FE
:1015E000D9CB83C75400A30CF40283C75400C1C7EE
:1015F00083C76400230DF40283C76400ADCF83C7A3
:101600007400A30DF40283C77400B5C783C78400B8
:10161000230EF40283C78400B9CF83C79400A30EBE
:10162000F40283C79400A1CB83C7A400230FF40264
:1016300083C7A400A9C383C7B400A30FF40283C760
:10164000B40095CB83C7C4002300F40483C7C4004F
:101650009DC383C7D400A300F40483C7D40081CF03
:1016600083C7E4002301F40483C7E40089C783C768
:10167000F400A301F404930A44005685A301040472
:101680002326340323283405232A0404EFE07FE9CA
:1016900013058401EFE0FFE8A947B3873741232C06
:1016A000040400C81CCC40D023220404232E0404CC
:1016B0005E86DA854A85EFE0FFE108C063040A0030
:1016C00023208A007370043017F90100130989E799
:1016D0008327090097F40100938484E891C7984018
:1016E0009C407C4385077CC317F70100130747E63E
:1016F0001C43850797F6010023ACF6E49C40C5CB5C
:101700008327090017FB0100130B8BF789EB9C4023
:10171000DC5763E6F90097F7010023A387E497F706
:101720000100938727E19C4317F701001307C7E1E6
:1017300048541843850797F6010023ADF6DE3CC4F4
:101740006376A70097F7010023A0A7E0D145EF50EB
:10175000201BD6855A95EFE03FDD8327090081C71E
:101760009C40FC43B5E383270900054499C79C408E
:10177000DC5763F43701EFE07FC92285B250225471
:1017800092540259F249624AD24A424BB24B4561E5
:1017900082805685EF20D0277D54C5B713152600CB
:1017A000EF20F014AA8AE31605DC7D54F9B797F709
:1017B000010023A787DA184385476301F70217FB67
:1017C0000100130BEBEBA1BF984094407C43FD1745
:1017D0007CC3FC42C9FB7360043071B7014A17FB3C
:1017E0000100130BEBE9A94B5285D145EF50401195
:1017F000050A5A95EFE0BFD1E3187AFF97FB010085
:10180000938B8BF45E85EFE09FD017FA0100130AEB
:10181000EAF45285EFE0BFCF17F50100130545F557
:10182000EFE0FFCE17F501001305C5F5EFE03FCE61
:1018300017F50100130545F6EFE07FCD97F701009E
:1018400023AE77D197F7010023A847D1C9BD411135
:1018500022C406C626C24AC02A847370043097F494
:101860000100938424CE9C40F9E311E497F7010032
:10187000938707CF8043130944004A85EFE05FCF89
:101880001C5489C713058401EFE09FCECA8517F564
:101890000100130525EFEFE03FC997F7010093879B
:1018A00067CB984397F701009387C7C89C43050708
:1018B00097F6010023A0E6CA9840850797F6010035
:1018C00023AAF6C601CB97F70100938767C998430F
:1018D000784349EF9C40B1C797F70100938747C809
:1018E0009843630F870873700430984039EB17F7FB
:1018F00001001307A7C614439442A5E27D5797F64B
:10190000010023A7E6C2984009CF9843784311CB42
:10191000984394437C43FD177CC3FC4299E3736076
:101920000430B2402244924402494101828097F738
:1019300001009387E7C298439C437C4385077CC39F
:101940002DB794439843F8420507F8C217F70100F2
:101950001307C7C014439442D5D218435847584779
:10196000584397F6010023A5E6BC71BF9843944302
:101970007C43FD177CC3FC42B1FF7360043099BF08
:1019800097F70100938787BA9C4381C7737004302F
:1019900001A02244B2409244024941016FE01FA7D6
:1019A00041C517F701001307A7BB14438147638B99
:1019B000A606411106C622C426C27370043097F6EB
:1019C0000100938626B89C4291C710431C437C4279
:1019D00085077CC29C42AA84404981C71C43FC43C2
:1019E000B9E797F70100938767B79C43638B870438
:1019F00097F70100938747B69C436384870497F762
:101A00000100938767D96309F40297F70100938770
:101A100067D76301F4028547B240224492443E8571
:101A2000410182803E8582807370043001A0EF50B6
:101A3000E00045BF9147CDB79C5493B71700890785
:101A4000E1BF8947D1BF7370043097F701009387D6
:101A500067AF984309EF15C59C43485581CB97F76D
:101A600001009387E7AF9843784315E3828017F727
:101A700001001307E7AE14431843F8420507F8C204
:101A800061FD17F701001307A7AD0843F1B79843AD
:101A900094437C43FD177CC3FC42E9FB7360043034
:101AA0008280411122C42A8406C6EFE01FA211E4FD
:101AB00097F701009387C7AA80434054EFE09FA0A7
:101AC000B2402285224441018280A54763F5B700D8
:101AD0007370043001A0011122CC06CE26CA4AC878
:101AE0004EC652C42A847370043017F901001309DA
:101AF00069A583270900CDEF71C43C486388F508C8
:101B000017F701001307C7A563FCB7001443638CE4
:101B1000860C18434457B3B4950093C4140029A00D
:101B20000443818C93B4140058546383E70A1C4C1B
:101B30002CC863C60700A947B385B7400CCC9317E0
:101B40002700BA97584897F90100938969B38A0723
:101B5000CE97631AF702130A44005285EFE05FA1A3
:101B600097F701009387479E48549C4363F6A7006C
:101B700097F7010023AAA79CD145EF407058D28562
:101B80004E95EFE07F9A99C0EFE05F8883270900C8
:101B900081CB97F701009387A79C9C43FC439DEB67
:101BA000F2406244D2444249B249224A05618280ED
:101BB00097F701009387C79A98439C437C43850716
:101BC0007CC305FC97F7010093878799804335B75D
:101BD0004CD4B1BF6244F240D2444249B249224A95
:101BE00005616F40B065814481B725C1011126CAE6
:101BF00097F401009384C4969C4006CE22CC4AC838
:101C00004EC6638DA7027370043017F901001309E3
:101C100069938327090091C798409C407C438507BE
:101C20007CC3584997F70100938707B76302F7020F
:101C30008327090081C79C40FC43A5EBF240624426
:101C4000D2444249B249056182807370043001A0D8
:101C50001C5517F701001307A7B1E38BE7FCE9FB5D
:101C6000930945002A844E85EFE09F9097F7010085
:101C70009387878D48549C4363F6A70097F701002C
:101C800023A4A78CD145EF40B04797F70100938775
:101C9000279F3E95CE85EFE03F899C405854DC5706
:101CA000E368F7F8EFE08FF661B76244F240D244A0
:101CB0004249B24905616F40705815CD011122CCDF
:101CC00026CA4EC62A8406CE4AC8EFE01F8058486E
:101CD00097F70100938747ACAA8981446300F70214
:101CE0004E85EFE02FFEF240624426854249D24401
:101CF000B249056182807370043001A01C5417F54D
:101D000001001305E5A6E38DA7FCF9FB97F7010099
:101D10009387C7819C43A9EB97F70100938747847A
:101D20009C43445413094400DC574A85B3B4F4007F
:101D3000EFE01F8497F701009387078148549C4385
:101D400093C4140063F6A70097E7010023AEA77EB3
:101D5000D145EF40F03A97F7010093876792CA8523
:101D60003E95EFE06FFCADBF93058401EFE0CFFB44
:101D700085BF0111056506CE22CC26CA4AC84EC6CB
:101D800052C456C25AC0EF208036630E051AAA8488
:101D900013050006EF20A0352A84630A051C05669A
:101DA0009305500A04D92685EF20A05A0458856768
:101DB000F117BE94B7474C4593879744130A4400E4
:101DC0005CD85285230C0402A301040423260402D8
:101DD00023280404232A0404EFE0AFF4130584014C
:101DE000EFE02FF4A947232C0404F19800C81CCC81
:101DF00040D023220404232E04040146971500003A
:101E00009385E5B12685EFE0EFEC08C073700430F0
:101E100017E90100130909738327090097E40100FA
:101E20009384047491C798409C407C4385077CC38D
:101E300017E701001307C7711C43850797E60100E8
:101E400023A8F6709C40C9C38327090097F90100B5
:101E50009389098381EB9C40DC5789E797E7010070
:101E600023A0877097E701009387C76C984397E694
:101E700001009386666D5C549442050717E60100E5
:101E8000232AE66A38C463F6F60017E70100232D1B
:101E9000F76A139527003E950A05D2854E95EFE027
:101EA000AFE88327090081C79C40FC43DDE7832717
:101EB000090091C39C40EF10F04985476305F50C7C
:101EC00059E17370043001A097E7010023AA8768E5
:101ED0001843854797E901009389897AE314F7F855
:101EE000CE8A17FB0100130B2B865685D10AEFE033
:101EF0000FE2E31C5BFF17F501001305E584EFE03B
:101F00000FE197FA0100938A6A855685EFE02FE08A
:101F100017F501001305C585EFE06FDF17F5010028
:101F200013054586EFE0AFDE17F501001305C58602
:101F3000EFE0EFDD97E7010023A2676397E7010079
:101F400023AC576105B7F2406244D2444249B249DA
:101F5000224A924A024B05618280984094407C4319
:101F6000FD177CC3FC42A1F77360043089B762445B
:101F7000F2404249B249224A924A024B2685D24453
:101F800005616F20E02873700430FD5717E70100EA
:101F90002320F75A624497E7010023A5A75AF2408D
:101FA000D2444249B249224A924A024B97E7010081
:101FB00023AE075805616FE0CFAE7370043097E72A
:101FC000010023A107586FE00FBC17E701001307BA
:101FD000E7551C4385071CC382807370043097E764
:101FE000010093872756984305E317E7010013077D
:101FF000E75508439C4381CB97E7010093874756F9
:102000009843784301EF828017E701001307475593
:1020100014431843F8420507F8C2C1BF98439443DC
:102020007C43FD177CC3FC42F9FF7360043082805F
:10203000411106C622C4EFE04FC997E7010093871C
:10204000E7508043EFE00FC8B240228522444101AF
:10205000828097E701009387A74F88438280797138
:1020600006D622D426D24AD04ECE52CC56CA5AC810
:102070005EC697E701009387674B9C43B1EF17E774
:1020800001001307A74C1C43850797E6010023AF07
:10209000F64A832A0700638F0A0697E701009387B1
:1020A00027499C43814463F1FA0897E90100938929
:1020B000295D17EA0100130AAA4A83270A00854608
:1020C000D85793172700BA978A07BE9983A70900A4
:1020D00063FFF600854421A897E7010093874746F0
:1020E0009C438144850717E70100232BF74497E7BA
:1020F00001009387A7449C4391C38544B250225466
:10210000268502599254F249624AD24A424BB24B56
:102110004561828017E40100130444441C409C4341
:10212000DDC37370043001A017E4010013040443FD
:1021300097E901009389C95417EA0100130A4A423A
:1021400017EB0100130B4B401C409C43B5C31C40D4
:10215000DC4703A9C70083274900930B49005E852C
:1021600063EEFA04EFE0CFC08327890213058901EB
:1021700099C3EFE0EFBF8327C90203270B00DE8579
:10218000139527003E950A054E956376F70017E7ED
:102190000100232BF73AEFE02FB983270A0003272A
:1021A000C902DC57E362F7FA1C4085449C43C5F33F
:1021B000FD5717E70100232DF73601B717E7010098
:1021C0002328F736DDBD17E701001307E7381C4069
:1021D000184397E6010023A3E63817E70100232DF3
:1021E000F73697E70100938727359C43850717E764
:1021F00001002323F7341C409C4399E7FD5717E760
:1022000001002327F73251BD1C40DC47DC47DC438B
:1022100017E70100232EF73049B597E701009387B0
:10222000E730984301E77370043001A0011106CE36
:1022300022CC26CA4AC84EC652C456C25AC073706F
:10224000043097E401009384E42F984061EB9843B5
:102250007D1797E6010023ABE62C9C43D9EB97E76B
:1022600001009387E72E9C43C9C797EA0100938A30
:102270002A4117EA0100130A2A2D17E90100130960
:10228000292E854919A83385EA00EFE0EFA98327B5
:1022900009005854DC576379F70483A70A0FC1CFAC
:1022A00083A7CA0FC04713058401EFE06FAC130B7F
:1022B00044005A85EFE0CFAB5C5483260A00DA85F0
:1022C000139527003E950A052A875695E3FDF6FAF1
:1022D00017E70100232AF726EFE00FA5832709005F
:1022E0005854DC57E36BF7FA97E7010023A837252A
:1022F0006DB701449C4081CB97E701009387472647
:102300009C43FC4395E72285F2406244D244424913
:10231000B249224A924A024B0561828017E70100C6
:102320001307072414431843F8420507F8C205B7FA
:10233000EF40C070C9BF17E40100130464201C40C3
:1023400095C31C40054999CF193B09C597E7010082
:1023500023A6271F1C40FD1717E701002322F71EA5
:102360001C40FDF397E701009387471D984385477D
:10237000E311F7F8EFE08F890544ADBF11CD81E59A
:102380007370043001A017E701001307271A1C43DC
:1023900099C77370043001A07370043001A041111B
:1023A00022C406C614431841850617E60100232FF0
:1023B000D61697E601009386661994423304B70057
:1023C00000C163F7E602637FE40063FD860097E7E0
:1023D00001009387E71888431105EFE06F99228584
:1023E000EF40805F1D3D01C9B2402244410182801F
:1023F000E36FE4FCD9BF2244B24041016FE00F819A
:1024000011C917E70100130767121C4391C77370C6
:10241000043001A06FD09FFF411106C622C41843AB
:10242000AA87050797E6010023A2E61097E60100B8
:102430009386061317E701001307471118438842D4
:102440003304F7001105EFE0AF922285EF40C0584A
:10245000E93311E52244B24041016FD03FFBB24065
:10246000224441018280411122C406C697E701003F
:102470009387C70B9C430144850717E70100232777
:10248000F70A97E701009387A70C9C4363E0F512D6
:1024900017EE0100130E8E2A97E201009382821D2F
:1024A00001440147854F1303500A21A0311E638D5B
:1024B000C20B83278EFFBA86F5DB8327CEFFDC4372
:1024C000232EFEFE638AC70F03AFC700DC432A97A3
:1024D000814E232EFEFE6385C70783A8C70093871E
:1024E0004803232017015CC383A788042326F70130
:1024F0001CC783A7C8021CCB83A70805232C070091
:102500005CCB03A808038347080063906704C28775
:10251000850783C60700B3850741E38B66FE898183
:10252000C205C181231EB700850E1307070263068B
:102530001F038327CEFFDC43232EFEFEE39FC7F954
:1025400083274E00232EFEFE49BF8145231EB70080
:10255000850E13070702E31E1FFD76941317540020
:10256000311EBA86E397C2F597E70100938707FF0C
:1025700003AE070083270E00639D070E97E7010057
:10258000938787FD03AE070083270E006392071829
:1025900017EE0100130ECE0E83274E109DE3832706
:1025A0008E116395072019C223200600BD312285B4
:1025B000B24022444101828083274E00232EFEFE3A
:1025C00021B783278E1017EF0100130F2F1CDC4358
:1025D00017E70100232AF71A6380E73383A2C700B5
:1025E000DC43AA96814E17E70100232FF718914F7D
:1025F0001303500A6388E70783A8C700938748033B
:1026000023A01601DCC283A7880423A6F6019CC67A
:1026100083A7C8029CCA83A7080523AC0600DCCAAE
:1026200003A80803834708006391672AC2878507C8
:1026300003C70700B3850741E30B67FE93D7250067
:10264000C207C183239EF600850E93860602638629
:10265000122983278E10DC4317E701002326F71287
:10266000E39CE7F983270E1117E70100232EF710EB
:1026700061B783274E00130F8E00D4432322DE0060
:102680006388E629B307E500D84283A2C600814EDD
:102690002322EE00894F1303500A6306EF068328B6
:1026A000C7001387480323A01701D8C303A78804D2
:1026B00023A6F70198C703A7C80298CB03A708056C
:1026C00023AC0700D8CB03A808030347080063180E
:1026D000671C4287050783460700B3050741E38B64
:1026E00066FE13D7250042074183239EE700850E2F
:1026F00093870702638D121B83264E00D842232244
:10270000EE00E31EEFF80327CE002322EE0041BFC8
:1027100083274E00130F8E00DC432322FE006384C8
:10272000E71F83A2C700DC43AA96814E2322FE0046
:10273000894F1303500A6306FF0683A8C7009387D7
:10274000480323A01601DCC283A7880423A6F60150
:102750009CC683A7C8029CCA83A7080523AC0600B1
:10276000DCCA03A808038347080063966710C28782
:10277000850703C70700B3850741E30B67FE93D7BF
:102780002500C207C183239EF600850E93860602AC
:10279000638B120F83274E00DC432322FE00E31ECF
:1027A000FFF88327CE002322FE0041BF8327CE11EE
:1027B00097EE0100938ECEFEDC4317E70100232F36
:1027C000F7FC6384D71383AFC700DC433307D5001E
:1027D000014397E6010023A3F6FC0D4F89429308BD
:1027E000500A6387D707C8479307450308C35CC3EC
:1027F0003C452326E7011CC75C551CCB1C5599C3DF
:10280000232657003C49232C07005CCB03280503F3
:102810008347080063951705C287850783C60700AD
:10282000B3850741E38B16FF93D72500C207C18309
:10283000231EF700050313070702638AAF028327ED
:10284000CE11DC4397E6010023AAF6F4E39DD7F905
:1028500083274E1297E6010023A2F6F469B7814759
:10286000231EF700050313070702E39AAFFC1A942F
:10287000E31C06D225BB8147239EF600850E938676
:102880000602E39912F117EE0100130E6EDF8327A3
:102890004E10769493165400E38307D01DB301477E
:1028A000239EE700850E93870702E39712E597E7DB
:1028B0000100938767CA03AE07007694931654000D
:1028C00083270E00E38607CCA1B58147239EF6003F
:1028D000850E93860602E39E12D783278E11769487
:1028E00093165400E38107CCD1B583274E1217E726
:1028F00001002325F7EAC1BD83270E1117E7010068
:102900002324F7E8E1B98327CE002322FE0011BD7E
:102910008326CE002322DE00B5B3797126D24AD0B9
:102920004ECE52CC56CA5AC85EC606D622D497E9B5
:1029300001009389A9BF17E90100130969D417EAB7
:102940000100130A2AC097EA0100938A6AC197EB33
:102950000100938BEBBF97E401009384A4BF054B68
:1029600021A883A7090003244910850717E7010060
:10297000232EF7BA5D3011E89C40E5F78327090064
:10298000E37CFBFEEFD09FA8C5BF737004308327A4
:102990000A00B9E383270911C04713054400EFD0AB
:1029A0003FBD83A70B00FD1717E701002322F7BAED
:1029B0009C40FD1717E70100232EF7B883270A0074
:1029C00089C783A70A00FC4385E30858EF10500429
:1029D0002285EF10F0034DB703A70A0083A70A0072
:1029E0007C4385077CC37DB703A70A0083A60A0042
:1029F0007C43FD177CC3FC42E9FB73600430F1B7F4
:102A000097E70100938787B29C43DDE7411106C633
:102A100022C426C297E7010023A207B217E70100EC
:102A2000130707B41C43B7A6A5A59386565A9C5B0B
:102A30008C43639BD500D0436318B60094476395DD
:102A4000C600DC476388D70008430C4393854503E1
:102A5000EF20007917E70100130707AF144317E4CD
:102A600001001304E4C111A81C43A9CF1C43FD17A6
:102A700097E6010023AAF6AC144393972600B69775
:102A80008A07A2979C43EDD3084393172500AA9782
:102A90008A073307F4005443A107A297C44244C3F2
:102AA0006385F402DC44B240224417E70100232985
:102AB000F7AA924441018280854717E70100232F3E
:102AC000F7A682807370043001A0C440D145EF3076
:102AD0003063229544C1F9B701114AC806CE22CC11
:102AE00026CA4EC62A897370043097E40100938485
:102AF00064A59C4017E40100130484A6D9E763147D
:102B0000090003290400930949004E85EFD05FA610
:102B10008327890289C713058901EFD07FA5CE8558
:102B200017E50100130545C7EFD01FA09C4081C7E2
:102B30001C40FC43ADE31C40638B27079C409DCFAA
:102B4000737004309C40C1EB97E70100938707A1A5
:102B50009843184325EBFD5717E70100232AF79CFC
:102B60009C4089CF1C40FC4391CB184014407C43CF
:102B7000FD177CC3FC4299E373600430F240624469
:102B8000D2444249B2490561828018401C407C43CE
:102B900085077CC3ADB7184014407C43FD177CC348
:102BA000FC42D1FB736004301C40E39927F99C4040
:102BB000A1C397E70100938767979C43ADCB7370E0
:102BC000043001A09C43DC47DC47DC4317E70100ED
:102BD0002320F79671B718401C407C4385077CC3BF
:102BE00097E7010093878797984318432DD7D9BF5C
:102BF00097E701009387C79517E70100130747A8D8
:102C00009C4303278711631DF700F240624497E756
:102C1000010023A70794D2444249B249056182804A
:102C20006244F240D2444249B2490561D1BB624498
:102C3000F240D2444249B24905616FD02FFD3DC9EF
:102C4000411126C297E40100938484914AC02E89E1
:102C50008C4006C622C4E105EFD09F8E8840110546
:102C6000EFD01F91FD57630AF90497E7010093879E
:102C7000E78D804398409C434A9440C3636CF404BE
:102C800097E701009387878D88438C409105EFD0AB
:102C90003F8B97E701009387A7899C436376F400F5
:102CA00097E7010023A68788B24022449244024954
:102CB000410182807370043001A08C402244B240F4
:102CC0009244024917E50100130505AD9105410144
:102CD0006FD09F8597E70100938707888843224438
:102CE0008C40B24092440249910541016FD05F850A
:102CF00011C997E70100938767839C4399E7737035
:102D0000043001A07370043001A0411126C297E481
:102D100001009384E4849840AE878C40B70600801D
:102D2000D58F06C622C41CCFE1053284EFD0CFFF79
:102D300088401105EFD0DF83FD57630EF40097E75D
:102D400001009387A7808843B24092442295224491
:102D500041016F3070488C402244B240924417E5E4
:102D60000100130565A3910541016FD0EFFB25CD4F
:102D7000411126C297D401009384847E4AC02E89D3
:102D80008C4006C622C4E1053284EFD0EFF98840BA
:102D90001105EFD0EFFD8547630AF40497D70100D2
:102DA0009387C77A804398409C434A9440C3636C9E
:102DB000F40497D701009387677A88438C40910584
:102DC000EFD00FF897D70100938787769C436376FF
:102DD000F40097D7010023AD8774B2402244924497
:102DE0000249410182807370043001A08C4022446A
:102DF000B2409244024917E501001305E599910597
:102E000041016FD06FF297D701009387E774884331
:102E100022448C40B24092440249910541016FD056
:102E20002FF2411106C622C426C25C45C04735CCEC
:102E3000930484012685EFD0AFF397D701009387E1
:102E4000E76E9C43B5E7930444002685EFD04FF22C
:102E500097D701009387476F58549C4363F6E70068
:102E600097D7010023A2E76E93172700BA978A0726
:102E700017E501001305C580A6853E95EFD0CFEA82
:102E800097D701009387C76D9C4358540145DC5781
:102E900063F8E700854717D701002321F76A054546
:102EA000B24022449244410182807370043001A0F8
:102EB000A68517E501001305A58BEFD0EFE6C9B78E
:102EC00097D70100938787669C4381E7737004302E
:102ED00001A0411106C622C426C2B70700804045A2
:102EE000CD8F1CC12DC4EFD0AFE8930444002685DC
:102EF000EFD00FE897D701009387076558549C439C
:102F000063F6E70097D7010023A0E7649317270033
:102F1000BA978A0717D50100130585763E95A685D1
:102F2000EFD08FE097D70100938787639C43585475
:102F30000145DC5763F8E700854717D70100232FC9
:102F4000F75E0545B240224492444101828073708D
:102F5000043001A011CD97D701009387E75D984316
:102F600097D701009387875E9C4318C15CC182801C
:102F70007370043001A055C1D1CD411106C622C4E1
:102F80002A877370043097D801009388A85B83A7C1
:102F9000080091CB97D701009387875C94439C43AB
:102FA000FC428507FCC217D301001303235A9C413E
:102FB00003260300FD560144638FD70217DE01008C
:102FC000130E8E5703250E00032807005443630594
:102FD000A80005446371D6023308D6400544637CDB
:102FE000F80003250E00918F03260300B6979CC1BD
:102FF00008C350C3014483A7080081CB97D70100C1
:10300000938707569C43FC4381EF2285B2402244BC
:10301000410182807370043001A07370043001A0FC
:10302000EF30D021DDB7854717D701002328F750AF
:10303000828019C1684582800145828011C16CC5BA
:10304000828097D701009387A7518843828097D7C2
:1030500001009387274F9C43054589CB97D70100F3
:103060009387C74C8843133515000605828031CD00
:10307000011126CA97D401009384844E9C4006CE49
:1030800022CC4AC84EC65855DC576379F7021C4D0E
:1030900063C707009C40D457A947958F1CCD931751
:1030A0002700BA97584917D901001309695D8A07A3
:1030B000CA97630DF7009C40DC575CD5F240624430
:1030C000D2444249B2490561828082809309450019
:1030D0002A844E85EFD0CFC99C4017D70100130733
:1030E000A7461843DC575CD46376F70017D7010076
:1030F000232CF744139527003E9562440A05F240BD
:10310000D244CE854A95B249424905616FD0CFC1BC
:1031100019CD411106C622C426C297D70100938754
:10312000274480436307A4007370043001A0014565
:1031300082807C4881E77370043001A05454384881
:10314000FD177CC86383E60099C70145B24022445D
:10315000924441018280930444002685EFD04FC100
:10316000284897D701009387273E9843A947898F1E
:1031700048D41CCC6376A70097D7010023A6A73CB0
:10318000D145EF30E07797D701009387674F3E95A1
:10319000A685EFD06FB9054555BF7370043097D73A
:1031A00001009387273A9C4391CB97D701009387DF
:1031B000273B98439C437C4385077CC3828097D7F9
:1031C0000100938727389C438DC397D701009387CD
:1031D00027399843784311CB984394437C43FD1798
:1031E0007CC3FC4299E373600430828097D701006E
:1031F00093870737904394439843A947D456084E82
:10320000958F1CCF828097D70100938767359843AD
:1032100009C79443F84A0507F8CA88438280797140
:103220004AD006D622D426D24ECE2A8973700430D4
:1032300097D40100938404319C4017D401001304F7
:103240002432BDE31C40BC4F89E71C400547F8CF42
:10325000D1E19C4081C71C40FC43F1EB737004300A
:103260009C408DEF1C40A84F11C5630409021C400F
:1032700023AC07041C4023AE07049C4081C71C40BC
:10328000FC438DEBB250225492540259F2494561ED
:10329000828018403C4FFD173CCFE9BF18401C40CE
:1032A0007C4385077CC37DBF18401C407C43850759
:1032B0007CC349BF184014407C43FD177CC3FC42CB
:1032C000F1F373600430B250225492540259F2491F
:1032D0004561828008402EC61105EFD06FA9B24526
:1032E000FD576380F50697D701009387272683A9AA
:1032F000070018409C43AE992322370163ECF90480
:1033000097D701009387872588430C409105EFD01C
:103310002FA397D701009387A7219C4363F6F90059
:1033200097D7010023A63721EFD04F8E1DB7184045
:1033300014407C43FD177CC3FC428DF37360043062
:1033400031BF0C4017D50100130505459105EFD09D
:10335000AF9DD9BF97D701009387072088430C40C2
:103360009105EFD0EF9DC9B779714AD04ECE06D600
:1033700022D426D252CC2E89B2897370043097D4CD
:1033800001009384241C9C4017D401001304441DA5
:10339000F9EF18408947784F630CF7001C4013453C
:1033A000F5FFB84F798DA8CF1C400547F8CFADE6A3
:1033B0009C4081C71C40FC43F5E3737004309C4083
:1033C000B1E7638609001C40BC4F23A0F9001840F8
:1033D00085470145784F630BF7001C401349F9FFFF
:1033E0000545B84F3379E90023AC27051C4023AECF
:1033F00007049C4081C71C40FC43C1E3B2502254E7
:1034000092540259F249624A4561828018401C4038
:103410007C4385077CC375B7084036C61105EFD0DD
:103420002F95B246FD576385F60897D7010093871D
:10343000E71103AA070018409C43369A232247014C
:103440006363FA0897D701009387471188430C40BC
:103450009105EFD0EF8E97D701009387670D9C43BE
:103460006370FA0697D7010023A4470D91A818406E
:103470001C407C4385077CC329BF184014407C4313
:10348000FD177CC3FC42BDFB73600430B250225474
:1034900092540259F249624A4561828018401440B0
:1034A0007C43FD177CC3FC4289FB7360043031B759
:1034B0000C4017D501001305252E9105EFD0CF86BE
:1034C000EFC0DFF4F5B597D701009387E70888438D
:1034D0000C409105EFD0CF86E5B751C1411106C62A
:1034E00022C426C24AC07370043097D4010093846A
:1034F00064059C40B9EB99C23C4D9CC2B287894699
:10350000704D74CD2E872A846386D70663FCF6043B
:103510008D456387B70091456395B7006300D60C6E
:1035200038CC8547630FF60405449C4081CB97D780
:1035300001009387E7029C43FC43A9E32285B24044
:103540002244924402494101828097D70100938727
:10355000270198439C437C4385077CC369BF7370F4
:10356000043001A08546E39ED7FA3C4D33E7B7000F
:1035700038CD45BF3C4D85073CCD65B7EF30004C9D
:1035800075BF130944004A85EFC09FFE97D701001D
:10359000938787FB48549C4363F6A70097D70100A5
:1035A00023A4A7FAD145EF30A03597D70100938720
:1035B000270D3E95CA85EFC03FF71C5481C7737035
:1035C000043001A097D70100938787F99C43585492
:1035D000DC57E3FBE7F4EFC07FE3B9B70144B1B7D1
:1035E00039CD011122CC26CA4AC84EC652C456C291
:1035F00006CEBA89368AB2842E892A84EFC0FFECBF
:10360000AA8A63050A003C4C2320FA00784C8947BB
:103610007CCC6389F40263F4970C8D466387D400F5
:1036200091466396D400630AF70A232C2405854744
:10363000631EF7061C5499CB7370043001A073709D
:10364000043001A03C4C85073CCCD5B797D701008E
:103650009387C7ED9C43ADEB930444002685EFC0F0
:103660003FF197D70100938727EE48549C4363F6B8
:10367000A70097D7010023A9A7ECD145EF30402838
:1036800097D701009387C7FFA6853E95EFC0DFE976
:1036900097D701009387C7EC9C435854DC5763F7D6
:1036A000E70063850900854723A0F9000544568596
:1036B000EFC05FE12285F2406244D2444249B24900
:1036C000224A924A056182809305840117D5010040
:1036D0001305050AEFC05FE565BF0144C9BF854713
:1036E000E397F4F43C4C33E92701232C240581B7FC
:1036F0004DC1011122CC26CA2A844EC606CE4AC824
:10370000AE84EFC09FDC8947744C7CCC3C4C0547B1
:10371000AA8985073CCC6395E6061C5481C7737063
:10372000043001A097D70100938747E09C43ADE7A1
:10373000130944004A85EFC0BFE397D70100938780
:10374000A7E048549C4363F6A70097D7010023AD38
:10375000A7DED145EF30C01A97D70100938747F213
:10376000CA853E95EFC05FDC97D70100938747DF9E
:103770009C435854DC5763F5E70099C085479CC0CB
:103780006244F240D24442494E85B24905616FC05D
:103790007FD37370043001A09305840117D5010015
:1037A000130505FDEFC05FD8C1B7AA8729C573709F
:1037B000043017D701001307E7D814439DE2F04FF8
:1037C000894601456315D60023AE070405451C4311
:1037D00081CB97D701009387A7D89843784315E307
:1037E000828097D601009386A6D790429442744275
:1037F000850674C2E9B797D70100938767D69C43C3
:103800007DB7984394437C43FD177CC3FC42E9FB9E
:103810007360043082805D71A6C2CAC052DC56DA81
:103820005AD85ED686C6A2C44EDE62D466D26AD0AC
:1038300017D901001309C9D317DB0100130B8BD271
:1038400097D40100938444D297DA0100938A0AD274
:10385000054AA54B83270900984363010712DC47FB
:1038600083A90700EFE06FF6EFE02FF783270B0047
:103870002A8C6362F50A97D7010023A5A7CE0146DB
:103880006370351B8840B3858941EFD07FA2EFE09C
:10389000DF98630105128840814601462C00EFD075
:1038A000CFDB4DD9A247E3C807FEC24983A7490130
:1038B00089C713854900EFC0BFCBEFE00FF2832724
:1038C0000B002A8C636DF508A24717D70100232B44
:1038D00087C9E3E2FBFCB317FA0013F70721631A69
:1038E000071613F7770C6318071E93F70702C5D75F
:1038F0004E85EF00F01145B7DC47C04783AC0700A9
:10390000930944004E85EFC0BFC65C502285829764
:103910005C4C6384470B83270900984371FF03A71E
:103920000A0097D6010023AF86C397D6010023AFC4
:10393000F6C297D7010023ADE7C2EFE01F8EA1BF0B
:10394000DC47C04703AD0700930C44006685EFC019
:103950003FC25C50228582975C4C6386470983276F
:103960000900984371FF03A70A0097D6010023AF0F
:10397000F6BE97D7010023ADE7BEB9B7EFE0EFE49D
:10398000EFE0AFE583270B002A8CE366F5F883A709
:103990000A00884081499043B385894117D70100C7
:1039A000232287BD13361600EFD09F90EFE0FF86ED
:1039B000E31305EEEFC09FA5F9BD1C4CCE85E6973D
:1039C00063E9FC049C4089CF02CA66CC22CEEFF0AA
:1039D0000FE88840814601464C08EFD0EF8705FD8F
:1039E0007370043001A01C4CE685EA97636CFD04FB
:1039F0009C4089CF02CA6ACC22CEEFF04FE58840C6
:103A0000814601464C08EFD02F8531F973700430A0
:103A100001A0032509005CC000C8EFC07FB2E5BD6E
:103A2000EFE0AFFF83270900DC47C047930C440059
:103A30006685EFC0FFB35C4C638F47035C50228503
:103A4000829791BD032509005CC000C8EFC05FAF3D
:103A500039B7B24723ACF900A5CFE29723A2F9000A
:103A600023A8390193854900636FFC0403A50A006C
:103A7000EFC01FAD0DB51C4C00C83387F90058C00E
:103A8000636DEC02330C3C416363FC029C4089CFC4
:103A900002CA4ECC22CEEFF08FDB88408146014631
:103AA0004C08EFC07FFB59F97370043001A003A5E7
:103AB0000A00E685EFC0DFA851B703250900E685B7
:103AC000EFC01FA8A5BF03250900EFC07FA7E1B382
:103AD0007370043001A0B24783A6890123A839017D
:103AE0003387D70023A2E9006364EC04B307FC40EA
:103AF00063EBD70483A749024E85829783A7C90148
:103B0000E39B47D983A68901B2479840B69711CF66
:103B100002CA3ECC4ECEEFF08FD38840814601469C
:103B20004C08EFC07FF3E31805D67370043001A092
:103B30006374FC00E370F7FC0325090093854900DA
:103B4000EFC01FA089BB03A50A0093854900EFC001
:103B50003F9F91B3411122C406C626C24AC017D462
:103B60000100130464A0EFF04FE31C4095CBEFF08D
:103B70000FE51C409DC381480148814709478146A4
:103B80001306004097D50100938545831705000073
:103B90001305A5C8EFD05F9A39E97370043001A00E
:103BA00017D90100130989C04A85EFC05F9697D4E1
:103BB00001009384E4C02685EFC07F950146B1459E
:103BC000114597D7010023A5279B97D7010023AF65
:103BD0009798EFC0FFC217D701002327A79811CDF0
:103BE00097C501009385057DEFD04FE149B7B240FD
:103BF000224492440249410182807370043001A042
:103C0000A5C9797156CAAA8A1305C00222D426D240
:103C10004AD04ECE52CC06D65AC85EC63A89B6892C
:103C2000328AAE84E9212A8405C9EFF00FD797D7ED
:103C30000100938767939C439DCFEFF04FD8130506
:103C400044002320540104CC232E440123203403B8
:103C500023222403EFC0FF8C2285B25022549254B9
:103C60000259F249624AD24A424BB24B45618280C4
:103C70007370043001A097DB0100938B2BB35E853A
:103C8000EFC0FF8817DB0100130B8BB35A85EFC021
:103C90001F880146B145114597D7010023AA778DAA
:103CA00097D7010023A4678DEFC09FB517D70100F8
:103CB000232CA78A01C997C501009385A56FEFD072
:103CC000EFD3A5BF7370043001A039C5011122CC18
:103CD00006CE26CA17D401001304048983280400E1
:103CE0002A88014563850802BA842EC2368732C409
:103CF00042C6954663C5B602EFF06FB58947630BC0
:103D0000F5020840814601464C00EFC0FFD4F24066
:103D10006244D244056182807370043001A04C007B
:103D200081463A864685EFC09FF5F2406244D24410
:103D3000056182800840814626864C00EFC0DFD1B5
:103D4000F9B719C1084182807370043001A001E500
:103D50007370043001A0411106C622C42A84EFF01A
:103D6000CFC348483334A000EFF06FC52285B2407E
:103D700022444101828001E57370043001A04111A9
:103D800022C42A8406C6EFF04FC10050EFF02FC3C3
:103D9000B240228522444101828001E573700430E3
:103DA00001A0411122C426C22E84AA8406C6EFF0C7
:103DB000CFBE80D02244B240924441016FF02FC068
:103DC0004111714522C406C61D262A8411C523202F
:103DD00005001105EFC0AFF32285B2402244410136
:103DE000828001CDB70700FFED8F81C7737004306B
:103DF00001A099E57370043001A07370043001A034
:103E0000011122CC4AC84EC652C456C206CE26CA9A
:103E1000BA893689B28A2E842A8AEFF04FA311E537
:103E2000638509007370043001A0EFE00F9A8324CA
:103E30000A00B37794006316090295C763870A00E6
:103E40009347F4FFE58F2320FA00EFE00FBDF24027
:103E5000624426854249D244B249224A924A0561C7
:103E60008280E30DF4FCE38209FEB3355001E205E4
:103E700063050900B7070004DD8D4E86C18D13056B
:103E80004A00EFE0FFE6EFE04FB919E1EFC00FD8CD
:103E9000EFF0CFB593176500AA8963D80700B70480
:103EA0000001FD14B3F499005DB7EFF00FAF832963
:103EB0000A00B3773401631E090089CB63880A00C6
:103EC0009347F4FFB3F737012320FA00EFF02FAF49
:103ED000F9B7E31DF4FEDDB701C9B70700FFED8FA9
:103EE00099C77370043001A07370043001A04111B0
:103EF00022C42A8406C626C24AC02E89EFF0EFA942
:103F000004409345F9FFB3F795001CC0EFF02FABC9
:103F1000B2402244268502499244410182804111E7
:103F200022C42A8406C6EFC04FDA0040EFC08FD902
:103F3000B240228522444101828009C9370700FF2F
:103F4000B3F7E50099C77370043001A073700430B3
:103F500001A06F207030B70700FFF18F81C7737029
:103F6000043001A001E67370043001A0011122CCDD
:103F70004AC84EC652C406CE26CA3689AE892A8A97
:103F80003284EFF0CF8C21E16305090073700430B7
:103F900001A0EFE08F8383240A00CE855285B3E42D
:103FA0009900613FB37794006307F40683240A0005
:103FB000EFE0AFA6F240624426854249D244B249BE
:103FC000224A05618280EFE04F8083240A00CE857B
:103FD0005285B3E434019537B3F78400638D8702CB
:103FE000E30609FCB70500054A86C18D13054A00A2
:103FF000EFE01FD0EFE06FA219E1EFC02FC1EFF0AB
:10400000EF9E93176500AA8463DF0700B7070001DE
:10401000FD17FD8C45B783270A001344F4FFE18F99
:104020002320FA0071B7EFF04F9783240A00B3778B
:104030009400639787009347F4FFE58F2320FA00ED
:10404000EFF0EF97E1B7411122C406C62A8426C2D9
:10405000EFD0BFF75C4085C308489304C4006316E3
:10406000950015A0084863009502B7050002EFE02F
:104070003FE55C40E5FB2285612A2244B240924440
:1040800041016FE08F997370043001A009C93707AF
:1040900000FFB3F7E50099C77370043001A0737097
:1040A000043001A06F20501B01C9B70700FFED8F3E
:1040B00099C77370043001A07370043001A04111DE
:1040C00022C426C206C62A84AE84EFF00F8D1840A3
:1040D00093C7F4FFF98F1CC02244B24092444101BF
:1040E0006FF0EF8D19C1084D82800145828041112A
:1040F00022C406C62A84EFD05FED97C701009387DC
:1041000067479C43A1EBE56717C701001307C76C1E
:10411000F11797C6010023A5E64617C70100232F14
:10412000F74417C70100232BF76A97C7010093874D
:10413000A74417C701002321F76A854717C7010065
:104140002322074417C701002328074217C701008D
:104150002322F74219E8EFE04F8CEF10E00701440B
:104160002285B24022444101828013058400937766
:104170003500C1EFE5671307F5FFE917E3EDE7FC4D
:1041800097C601009386C63F9C4229A0984311C759
:10419000BE86BA87D843E36BA7FE17C70100130793
:1041A000A73DE38AE7FA984341461384870098C203
:1041B000D843B306A7406378D6023388A7002322EA
:1041C000D800C8C38325480097C601009386463BA4
:1041D00011A0BA8698425043E36DB6FE2320E80052
:1041E00023A00601D84397C701009387673D9C43EE
:1041F000998F17C701002325F73CEFE00F8231DCD0
:104200002285B240224441018280719911059DB7F7
:1042100029C9411122C406C62A84EFD01FDB9305A9
:1042200084FF0326C4FF17C701001307673511A0D9
:104230003E871C43D443E3EDC6FE232CF4FE0CC39F
:1042400097C701009387C73798438327C4FF224449
:10425000B240BA9717C701002324F73641016FD047
:10426000DFFB828097C70100938787358843828070
:1042700082803367B5000D8BAA871DE79308D6FFB0
:10428000AA982A87AE866371150303A80600110752
:104290009106232E07FFE36A17FF9347F5FFC697A2
:1042A000F19B9107BE95AA972A9663F3C70A938656
:1042B000450013884700B3B6D70033B8050133E78C
:1042C000F50093C61600134818000D8BB3E60601DF
:1042D00013371700758F330EF6409386170029CFDA
:1042E0001337AE0031EB13532E002E88BE860147E4
:1042F000832808000507110823A016019106E36929
:1043000067FE1377CEFFBA95BA976302EE0483C6B1
:104310000500138717002380D700637AC70283C67E
:10432000150013872700A380D7006372C70203C755
:1043300025002381E7008280B307F640AE9785050C
:1043400003C7F5FF8506238FE6FEE39AF5FE82801C
:104350008280B367C5008D8BB308C500E9C3637164
:10436000150FB307A0408D8B13873700954693F543
:10437000F50F130815003383A8407D166373D7002B
:1043800015476363E60CD5CF2300B5000547638D61
:10439000E700A300B5000D47130825006396E7006A
:1043A000130835002301B500139685004D8E139731
:1043B0000501518F3303F34093968501D98E13562F
:1043C0002300AA97014794C305079107E36DC7FE31
:1043D0001377C3FFB307E8006307E3062380B70042
:1043E00013871700637C1703A380B7001387270088
:1043F000637617032381B7001387370063701703B1
:10440000A381B70013874700637A17012382B7009F
:104410001387570063741701A382B700828093F556
:10442000F50F13978500D98D139705014D8FE3770D
:1044300015FFAA87910723AEE7FEE3ED17FF828001
:1044400082802A8895B78280AA8749BF8347050062
:104450002A8799C7050583470500EDFF198D8280DE
:104460000145828005058347F5FF850503C7F5FFF4
:1044700091C7E389E7FE3385E74082808147E5BF46
:10448000AA87850503C7F5FF8507A38FE7FE75FBA0
:10449000828083460500930700026397F6000505B6
:1044A00083460500E38DF6FE938756FD93F7D70FFD
:1044B00085C7AA87814585CE01458507138606FDF8
:1044C0001317250083C607003A9506053295F5F6C1
:1044D00099C13305A0408280938536FD834615003F
:1044E00093B5150093071500E1FA0145D5B70145CD
:1044F00082809C412380A7009C4185079CC18280CB
:1045000097C60100938646089C421757030013077D
:10451000672F13861700BA972380A70097C501005D
:1045200023A4C506A9476308F500930700046305A3
:10453000F6000145828075DE370610F005078347D7
:10454000F7FF2320F6F09C42FD1797C5010023AD2D
:10455000F502EDF7014582804D712322911423204D
:104560002115232A511323248113232611142324D4
:104570008114232E3113232C411323286113232666
:104580007113232291132320A113232EB111AA8486
:104590002E8932C6130C5002A54A83470900638056
:1045A0008703B9CB804011A0A1CB2300F400804049
:1045B0000509050480C083470900E39787FF034688
:1045C000190093081900C686130D0002FD597D5A83
:1045D0000148130550059307D6FD93F7F70F13898C
:1045E00016006363F52A17C701001307A7A18A07FE
:1045F000BA979C43BA9782878320C11403248114FD
:1046000083244114032901148329C113032A81132C
:10461000832A4113032B0113832BC112032C811214
:10462000832C4112032D0112832DC11171618280EF
:10463000A14C02C4854763D50715B2478040938BD0
:10464000770093F68BFF03AB060083A946009387A0
:1046500086003EC6668681465A85CE85EF10505A42
:104660002AC8814763853723930D4101854B6686B0
:1046700081465A85CE85EF10E07A814666862A8B80
:10468000AE89EF10F057A24723A0AD0093861B0020
:10469000910D63843701B68BD9BFE37E9BFF63DD49
:1046A0004601A2872380A70180407D1A930714004A
:1046B0009CC03E84E3C846FF93962B001C08BE9620
:1046C00031A8938777052300F4008040FD1B938772
:1046D0001B00050480C0F116E351F0EC9C42E3E2BC
:1046E000FAFE93870703C5B79C4093060003324741
:1046F0002380D7009C4093064700C14C13861700C7
:1047000090C013068007A380C700804002C4BA8708
:10471000050480C003AB0700814936C625BFB247F8
:1047200083AC0700938B470063840C1C635F4019C4
:104730009307D0026319FD1683C70C0085C363DCA1
:1047400009189440850C7D1A2380F60080400504EA
:1047500080C083C70C00E5F7635D4001804093078C
:1047600000022300F40080407D1A050480C0E31A93
:104770000AFE5EC61DB502C48547A94CE3CF07EB10
:10478000B24780409386470071B703C61600CA86B9
:1047900099B59C40930650022380D70080400504C1
:1047A00080C0E5BBC14C02C471B5B24703C6160058
:1047B000CA8683A9070091073EC6E35E0AE04E8AD7
:1047C000FD5911BD03C61600130DD002CA8621B5CE
:1047D0009347FAFFFD8703C61600337AFA00CA86AC
:1047E000DDBB03C61600130D0003CA86EDB383C5F7
:1047F0001600930906FDCA86938705FD2E86E3EE13
:10480000FAFA93972900BE9985068609AE9983C561
:104810000600938909FD938705FD2E86E3F3FAFED2
:1048200069BF32479C40144311073AC62380D70022
:104830008040050480C095B3854763D3070BB2471A
:1048400093867700E19A938786003EC683A9460047
:104850009C4263DC090A94401306D002B307F0407F
:104860002380C6008040B336F000B3093041050410
:1048700080C03E8BB389D940A94C02C4E1BB03C6BA
:1048800016000508CA8681BB9C40468921B7E37D96
:104890009BDD8547814B8546E3C547E131BD97CC1C
:1048A0000100938C2CB2CE856685EF00F07F330A31
:1048B000AA40635C400180402300A40180407D1A2F
:1048C000050480C0E31A0AFE014A83C70C00E38294
:1048D00007EAE3C809E6FD197D57E394E9E6ADBDB3
:1048E000B247938647009C4336C693D9F74195B7A4
:1048F000635640019307D002E313FDFA97CC010001
:10490000938C4CAC930780021DBD3E8BA94C02C416
:10491000804089B34D71232E3113B709004093872E
:10492000F9FF2324811423229114232C4113232AD9
:104930005113232611142320211523286113232624
:10494000711323248113232291132320A113232ED7
:10495000B1112A8A2EC417C401001304E4C2975A65
:104960000300938A2AEA97B401009384247F3EC609
:1049700093055002294513080004B70610F0834739
:104980000A006386B704C1C71840050A130617005A
:10499000569797C8010023A9C8BE2300F700638279
:1049A000A706E31E06FD175703001307A7E5050733
:1049B0008347F7FF23A0F6F01C40FD1717C6010040
:1049C0002324F6BCEDF783470A00E39EB7FA83463B
:1049D0001A0013051A002A87930B00027D5B7D5C89
:1049E000014893055005A5489387D6FD93F7F70F27
:1049F000130A170063E7F5348A07A6979C43A69726
:104A00008287175703001307E7DF55F28DBF832016
:104A1000C11403248114832441140329011483291C
:104A2000C113032A8113832A4113032B0113832B00
:104A3000C112032C8112832C4112032D0112832DEC
:104A4000C11171618280A14C014D854763DB07195B
:104A5000A2479D07E19B83AD070003AB4700138787
:104A600087003AC4668681466E85DA85EF10501954
:104A70002AC863066D35130941018549668681465A
:104A80006E85DA85EF10003A66868146AA8D2E8BF8
:104A9000EF1010172320A90085091109E3106DFFFD
:104AA000E3FE9DFD13060004B70610F063D18903F1
:104AB0001C4013871700D69797C5010023A6E5ACC5
:104AC00023807701630CC7047D1CE3C389FFB247D1
:104AD0006800A548B386F9008A061C08BE962948D6
:104AE00013030004370610F0E384A6E89C42930504
:104AF000000363F4F800930570051840AE97930522
:104B00001700569717CE01002320BEA82300F700F8
:104B10006380072B638C6526F116F9B717570300DE
:104B2000130747CE05078347F7FF23A0F6F01C4085
:104B3000FD1797C5010023A9F5A4EDF77D1C71B7FA
:104B40001C40130600041387170097C5010023AD0E
:104B5000E5A2B386FA00930500032380B600630044
:104B6000C73E890797C6010023A0F6A25697930671
:104B700080072300D700175703001307A7C8B706FD
:104B800010F0639EC70005078347F7FF23A0F6F0E8
:104B90001C40FD1717C601002328F69EEDF7A2471B
:104BA000C14C014D91072247014B832D07003EC4A4
:104BB00055BDA24783AC070013894700638F0C3AA9
:104BC000635480219307D002639EFB2E03C70C0021
:104BD000BA856310072025AC8547A94C014DE3C970
:104BE00007E7A2479107C1B7A2478346170052873C
:104BF00003AB070091073EC4E3580CDE5A8C7D5B83
:104C0000E5B383461700930BD0025287F1BB93475D
:104C1000FCFFFD8783461700337CFC005287E9B315
:104C200083461700930B000352877DBB0346170092
:104C3000138B06FD5287930706FDB286E3EEF8FA62
:104C400093172B00DA9705078607B29703460700EC
:104C5000138B07FD930706FDB286E3F3F8FE69BFE9
:104C6000A2451C402946984193861700D69717C540
:104C70000100232BD5902380E700138945006301B1
:104C8000C72A930700046387F6204AC4D5B1854735
:104C900063DF0729A24713877700619B930787008B
:104CA0003EC4032B47001C43635B0B3018401306C4
:104CB00000049306170097C5010023A7D58C5697CB
:104CC0009305D0022300B7006388C62CB307F040D9
:104CD0003337F000330B6041BE8D330BEB40A94CF2
:104CE000014D49B38346170005085287F5B983463D
:104CF00017005287D5B91C4093060004138717008C
:104D000017C601002322E688D69713065002238097
:104D1000C700E31FD7C4175703001307A7AEB70692
:104D200010F005078347F7FF23A0F6F01C40FD179E
:104D300017C60100232AF684EDF71DB9C14C014DB9
:104D400029B31C40930600042A8A1387170017C64C
:104D50000100232BE682D697130650022380C7005A
:104D6000E318D7C0175703001307C7A9B70610F0F9
:104D700005078347F7FF23A0F6F01C40FD1717C671
:104D800001002323F680EDF72A8ADDB617570300CA
:104D9000130747A705078347F7FF2320F6F01C40BA
:104DA000FD1797B5010023A1F57EEDF7F1162DBB98
:104DB00017570300130707A5F1FDF11635B3E3FC00
:104DC0009DCB8549C5B1014C03C70C00BA85E30EE4
:104DD00007EAFD58294513080004B70610F0635789
:104DE0000B0A1C4013861700D69717B30100232D1A
:104DF000C3782380E7006384A50663040609850C55
:104E000003C70C007D1CBA8579FBE35080E91C4088
:104E10009305000213060004B70610F021A07D1CC4
:104E2000E3050CE613871700D6972380B70017B564
:104E30000100232BE574BA87E313C7FE175703005D
:104E40001307479C05078347F7FF23A0F6F01C4094
:104E5000FD1717B501002329F572EDF7C9B71757EC
:104E600003001307279A41DE05078347F7FF23A0B6
:104E7000F6F01C40FD1717B601002327F670EDF77A
:104E8000BDBF175703001307E797F9BF7D1BE31A50
:104E90001BF5A5BF175703001307C796B70610F0F9
:104EA00005078347F7FF23A0F6F01C40FD1717B650
:104EB0000100232BF66CEDF74AC45DBC97BC0100E2
:104EC000938C4C50DA856685EF00101E330CAC4095
:104ED000E35C80EF1C4013060004B70610F021A02D
:104EE0007D1CE3020CEE13871700D6972380770111
:104EF00097B5010023AAE568BA87E313C7FE1757E1
:104F000003001307279005078347F7FF23A0F6F058
:104F10001C40FD1797B5010023A8F566EDF7C9B74A
:104F2000175703001307078EB5FA4AC491B4A24776
:104F3000138747009C433AC413DBF741B5B31757B7
:104F400003001307278CB70610F005078347F7FF08
:104F500023A0F6F01C40FD1717B601002326F662C9
:104F6000EDF7854717B701002320F7629307800705
:104F7000175703002308F7881DB163568001930774
:104F8000D002E39DFBF297BC0100938CAC43130766
:104F900080029305800235BD97560300938686866E
:104FA000370610F0850603C7F6FF2320E6F0184009
:104FB0007D1797B5010023A9E55C6DF701BBBE8D98
:104FC000A94C014D45B4B70710F023A0A7F201A0EA
:104FD0003971130341022ED29A8506CE32D436D6C9
:104FE0003AD83EDA42DC46DE1AC62D32F24001459E
:104FF000216182805D711303810322D42AC632DCD1
:105000002A841A86680006D6BEC236DEBAC0C2C47A
:10501000C6C61ACEEFF04FD4B24723800700324500
:10502000B250018D225461618280B70710F083A6CF
:1050300047F403A607F403A747F4E31AD7FE8566EF
:10504000938606FAB29633B6C600B305E60023A4EB
:10505000D7F423A6B7F48280B70710F003A747F46C
:1050600003A607F483A647F4E31AD7FE8566938662
:1050700006FAB29633B6C60023A4D7F4B305E60009
:1050800023A6B7F49307000873A04730828041112C
:1050900022C406C651447D143D2D75FCB240224405
:1050A00041018280411122C406C697B7010093874F
:1050B000274E17B401001304644D98431C40130697
:1050C000F07C930647069387470697B5010023A116
:1050D000D54C97B5010023ABF54A6346D600B240E4
:1050E0002244410182801307478997B7010023A119
:1050F000E74A052385476310F502184085679387C3
:10510000F7760145E3DDE7FCEFF0FFEB2244B24028
:1051100041016FC09FEA17B501001305252BEFF081
:105120003FEB0945EFF03FEA2244B24041016FC036
:10513000DFE817B501001305E52A6FF07FE917B521
:1051400001001305A52A6FF0BFE8411122C426C251
:1051500006C6856417B401001304C42993878438F4
:105160000100FD17F5FF2285EFF09FE6C5BF411155
:1051700006C622C4152917070000130787F18146C8
:1051800005469305200317B5010013052527EFE019
:105190003FA72A84EFC07FE42A8622852244B240BA
:1051A00001478146854541016FE03FB2411106C686
:1051B0008D21054781476316E500B2403E854101D8
:1051C000828017B5010013056520EFF07FE0B24043
:1051D00089473E85410182807370043001A082803E
:1051E0007370043001A05D71A6C2CAC04EDE52DCED
:1051F0008D69375AC6412169C164A2C456DA5AD8AA
:105200005ED662D46AD06ECE86C666D202C668000A
:1052100017BC0100130CCC39974B0300938B8B62A6
:1052200017BB0100130B4B3817BD0100130D8D3751
:10523000974D0300938D8D67130ADAE693899903DE
:105240007D190544FD14C54A894CD285EF10406B89
:10525000B307350113D5070117B70100232AF73427
:105260008D4533752501EF10E0700A05B387AB005B
:10527000D8478843814605077D566C00D8C7EFB0F4
:10528000AFFD6306850097B7010023A30734B2473B
:105290008507638B970403270B003EC6930717000F
:1052A00017B701002322F73063FAFA0483270D00B1
:1052B00017B70100232A072E63818706B9C3639FAE
:1052C0009703974703009387275E88438545EFC080
:1052D000CFFF1305800C97B7010023A5072CEFD053
:1052E0002F9203250C008DB783270B0002C685077C
:1052F00017B70100232AF72AE3EAFAFA03250C007C
:10530000A9B703A50D008145EFC02FFC03250C00B4
:1053100097B7010023A8872805BF03A50D00854581
:10532000EFC0AFFA9747030093870758884381453A
:10533000EFC0AFF9894717B701002325F7260325EA
:105340000C0019B73971254522DC26DA4AD84ED629
:1053500052D406DE56D25AD05ECE62CC66CA6AC835
:1053600002C6974403009384E44DEFC04F8597B77E
:10537000010023A5A7242689174A0300130A4A4DD2
:1053800017B40100130484238549014691450D4556
:10539000EFB00FC72320A900630A051C0C40EFC023
:1053A000CF8A630D351B97B7010023A3072211098C
:1053B000E31D49FD88408145EFC0AF8C09C597B713
:1053C000010023A707200C408840EFC08F8B854742
:1053D0006306F50097B7010023AC071E88406C00F8
:1053E00081460146EFB04FE70C408840EFC0EF85A3
:1053F00009C597B7010023AD071C884081460146C7
:105400006C00EFB09FA50C408840EFC00F8485472B
:105410006306F50097B7010023AC071A084093050F
:10542000800CEFC02F8909C597B7010023A2071A86
:1054300097470300938747478843C1644179EFC08A
:10544000CFFA85479389E4FF17BC0100130CCC17F2
:1054500017BA0100130ACA1717B70100232CF71453
:1054600097BB0100938B8B1417BD0100130DCD1456
:10547000054B954A994C0509FD140145EFC0AFDC79
:1054800039C90840FD55EFC0EF8221CD8146014664
:105490006C00EFB09F9C6306650197B7010023A9DC
:1054A0000712EFD09FCFB24763F2F9043387270189
:1054B00063FDEA006157636AF70003270C00637D10
:1054C000F70A998F0D476366F70A83270A00B5EB41
:1054D0007370043001A00840FD55EFB0BFFD5DF5CD
:1054E00069BF97B7010023A5070E41BF63FEFA000D
:1054F0003387F94063FAEC0003A70B006376F708E3
:10550000998F0D47636FF70883270A0081E773704F
:10551000043001A083A70B00850763FFF90697B746
:10552000010023A50708EFD09FC983270A00E3964F
:1055300067F583270D00850717B70100232EF706AF
:105540002DBF83270C00850717B70100232EF70610
:10555000F9FB97B7010023A99706F1B703250900C6
:105560000C40EFB09FEEE30405E435BD73700430EA
:1055700001A07370043001A0B307F7400D47E37634
:10558000F7F47370043001A0B307F7400D47E37DD3
:10559000F7F67370043001A017B701002328F70055
:1055A00059B77370043001A04111814801489747F1
:1055B00003009387672F054781461306004097B580
:1055C00001009385E5E417050000130505C206C632
:1055D00022C4EFB07FF6174403001304E42C1440F8
:1055E00081480148974703009387472C05471306D6
:1055F000004097B50100938525E2170500001305CB
:10560000A5D4EFB07FF308402244B24041016FD0EF
:10561000AFCC974703009387E72217B3010013032A
:10562000A3F983A8C700904F17B70100130747F7E6
:10563000032E0300084303A80701D44FCC4B985313
:105640003386C84097B70100938787F8832E0300FD
:105650003305C5419C433336C0003306C040B38692
:1056600006413335A000718DB336D0000D8F17B3CE
:1056700001001303A3F517B60100130626F2B306C3
:10568000D0403337E000FD17032E030010423307EC
:10569000E040758D93B71700798DB307F04017B7C9
:1056A0000100232FD7EF174703002329171B1747A4
:1056B00003002327071B174703002325B71A7D8DF7
:1056C0006309CE008327030017B701002328F7ECF6
:1056D000828001458280011197B70100938787ED91
:1056E00006CE22CC804385476306F400F240624434
:1056F0000561828097B70100938707EA9C431307EF
:1057000040068507636AF700F240624417B701005C
:105710002324F7E80561828097B70100938707EAA1
:10572000884397B7010023A907E6EFB01FDA25C524
:1057300001466C00EFB01F8D6306850097B701002E
:1057400023A807E8B24741677917637AF70A4177D8
:1057500005073E97954663F6E610615797B6010038
:10576000938686E66363F71098426379F710998F02
:105770000D47637CF70E7370043001A09C428507CF
:1057800017B701002322F7E499E7C167FD1717B7A0
:105790000100232BF7E217B401001304A4DF1C401F
:1057A000814601461397270097470300938787098F
:1057B000BA97884397B50100938545E1EFB02FCCA8
:1057C0008547E315F5F217B70100130727E01C43DF
:1057D000850797B6010023ABF6DE1C4399E7C16746
:1057E000FD1717B701002323F7DE1C400947850783
:1057F0006354F70697B7010023AE07D8C5BD954699
:1058000063F4F6021D8F994663F0E60297B6010035
:105810009386C6D99842637BF706998F0D476379C3
:10582000F7007370043001A097B60100938606D884
:1058300097B701009387C7D99C4381CF9C424167AA
:1058400079178507637CF70497B7010023A007D673
:1058500099B77370043001A017B70100232CF7D259
:1058600071B597B60100938626D697B70100938746
:1058700027D69C4381F77370043001A0B307F7402B
:105880000D47E374F7FE7370043001A0B307F740CF
:105890000D47E37FF7F87370043001A017B70100DC
:1058A0002326F7D0CDBD0000B305B5009307050052
:1058B0006386B70003C70700631607003385A74058
:1058C00067800000938717006FF09FFE130101FBB4
:1058D00023229104232C4103232291032326110424
:1058E0002324810423202105232E3103232A51035D
:1058F0002328610323267103232481032320A1038A
:10590000232EB101930C0500138A050093040000B7
:1059100063DE05003305A0403337A000B305B04077
:10592000930C0500338AE5409304F0FF63DA060028
:105930003306C040B337C000B306D040B386F6404C
:10594000930A06009389060013840C0013090A00C9
:105950006396062817BB0100130BCB956370CA161C
:10596000B70701006372F6149307F00F63F4C700E2
:1059700093098000B3573601330BFB0083470B00BC
:1059800013050002B3873701B309F540638C0900A2
:10599000B3153A01B3D7FC00B31A360133E9B700A7
:1059A00033943C0113DB0A0193050B001305090036
:1059B000EF00507C130A050093050B00939B0A012E
:1059C00013050900EF00907693DB0B0193050500AA
:1059D00013850B00EF00D072131A0A0193570401CC
:1059E000B367FA0063FAA700B387570163E657016C
:1059F00063F4A700B38757013389A74093050B00D1
:105A000013050900EF001077130A050093050B003A
:105A100013050900EF0090711314040193050500AC
:105A2000131A0A0113850B0013540401EF00506D83
:105A300033648A00637AA40033045401636654011A
:105A40006374A400330454013304A4403354340178
:105A500093050000638A040033048040B33780005C
:105A6000B305B040B385F540130504008320C1049D
:105A70000324810483244104032901048329C103ED
:105A8000032A8103832A4103032B0103832BC102D1
:105A9000032C8102832C4102032D0102832DC101BD
:105AA0001301010567800000B70700019309000199
:105AB000E362F6EC930980016FF0DFEB631A0600F6
:105AC0009305000013051000EF005066930A0500CF
:105AD000B707010063FAFA0E9307F00F63F457015A
:105AE00093098000B3D73A01330BFB0083470B00C7
:105AF0001305000233095A41B3873701B309F54052
:105B0000E38209EAB39A3A01335BFA00B3153A012A
:105B1000B3D7FC0093DB0A0133E9B70013050B0090
:105B200093850B00EF001065130A050093850B00A9
:105B3000139C0A0113050B00EF00505F135C0C016E
:105B40009305050013050C00EF00905B131A0A0182
:105B500093570901B367FA0033943C0163FAA70035
:105B6000B387570163E6570163F4A700B387570172
:105B7000338BA74093850B0013050B00EF00905F5C
:105B8000130A050093850B0013050B00EF00105A54
:105B90009305050013050C00EF00905693160901BC
:105BA000131A0A0193D60601B366DA0063FAA60057
:105BB000B386560163E6560163F4A600B386560128
:105BC0003389A6406FF01FDEB7070001930900017B
:105BD000E3EAFAF0930980016FF0DFF06376DA0010
:105BE00093050A006FF01FE7B707010063FAF60498
:105BF000930BF00F33B5DB001315350033D7A60038
:105C000097A701009387076BB387E70083CB070053
:105C100093050002B38BAB00338B7541631C0B0201
:105C200063E4460163EACC003384CC40B306DA4037
:105C300033B98C0033892641930509006FF09FE149
:105C4000B707000113050001E3EAF6FA1305800126
:105C50006FF0DFFAB3966601335D7601336DDD00D8
:105C6000B35D7A01B3156A0133DC7C0113540D0175
:105C7000336CBC0013850D0093050400B319660155
:105C8000EF00504F930A05009305040013850D00A3
:105C900033996C01931C0D01EF00504993DC0C010A
:105CA000130A05009305050013850C00EF0050450D
:105CB000939A0A0113570C0133E7EA00930D0A0087
:105CC000637EA7003307A701930DFAFF6368A7015E
:105CD0006376A700930DEAFF3307A701330AA740B5
:105CE0009305040013050A00EF00D0489305040053
:105CF000930A050013050A00EF00504393050500C1
:105D00001304050013850C00EF00903F93150C0160
:105D1000939A0A0193D50501B3E5BA00130704006D
:105D200063FEA500B385A5011307F4FF63E8A50191
:105D300063F6A5001307E4FFB385A501939D0D014C
:105D4000B70C0100B3EDED001384FCFFB3F78D0039
:105D500033F48900338AA5401385070093050400B6
:105D60002326F10093DD0D01EF0090399305040027
:105D7000930A050013850D00EF00903813DC09012C
:105D800093050C002324A10013850D00EF0050376C
:105D90008327C10013040C0093050400130C0500B5
:105DA00013850700EF00D0358326810013D70A0141
:105DB0003305D5003307A7006374D700330C9C016B
:105DC000B70701009387F7FF935507013377F70073
:105DD00013170701B3F7FA00B3858501B307F7007E
:105DE0006366BA00631EBA00637CF90033863741EC
:105DF000B3B7C700B385A541B385F5409307060047
:105E0000B307F9403339F900B305BA40B3852541EA
:105E100033947501B3D767013364F400B3D56501DA
:105E20006FF05FC3130101FD23229102232A510168
:105E3000232611022324810223202103232E310152
:105E4000232C410123286101232671012324810190
:105E5000232291012320A101930A050093840500C8
:105E6000639E0638130406009309050017A9010074
:105E70001309494463F8C512B7070100138B0500E5
:105E80006378F6101307F00F3337C7001317370086
:105E9000B357E6003309F900834609003387E6006B
:105EA00093060002B386E640638C0600B394D400E8
:105EB00033D7EA003314D600336B9700B399DA0076
:105EC000935A040193850A0013050B00EF00902AF2
:105ED0001309050093850A00931B040113050B00A9
:105EE000EF00D02493DB0B0193040500930505001C
:105EF00013850B00EF00D0201319090193D7090176
:105F0000B367F900138A040063FEA700B387870014
:105F1000138AF4FF63E8870063F6A700138AE4FF9F
:105F2000B3878700B384A74093850A0013850400D4
:105F3000EF0050241309050093850A00138504001F
:105F4000EF00D01E93990901930405009305050005
:105F50001319090113850B0093D90901EF00501A99
:105F6000B36939011386040063FCA900B309340145
:105F70001386F4FF63E6890063F4A9001386E4FF47
:105F800013140A013364C400130A00006F000013E5
:105F9000B707000113070001E36CF6EE1307800159
:105FA0006FF01FEF138A0600631A060093050000C6
:105FB00013051000EF00901713040500B707010048
:105FC000637EF4129307F00F63F48700130A8000D6
:105FD000B35744013309F90003470900930600024F
:105FE00033074701B386E64063940612B3848440C6
:105FF000130A1000135B040193050B0013850400C2
:10600000EF0050171309050093050B0013850400DA
:10601000931B0401EF00901193DB0B019304050027
:106020009305050013850B00EF00900D131909016E
:1060300093D70901B367F900938A040063FEA700B0
:10604000B3878700938AF4FF63E8870063F6A700AD
:10605000938AE4FFB3878700B384A74093050B00BE
:1060600013850400EF0010111309050093050B00C0
:1060700013850400EF00900B939909019304050028
:10608000930505001319090113850B0093D9090124
:10609000EF001007B36939011386040063FCA900FF
:1060A000B30934011386F4FF63E6890063F4A900A1
:1060B0001386E4FF13940A013364C400130504003B
:1060C00093050A008320C102032481028324410234
:1060D000032901028329C101032A8101832A410185
:1060E000032B0101832BC100032C8100832C410071
:1060F000032D01001301010367800000B7070001B1
:10610000130A0001E366F4EC130A80016FF05FEC00
:106110003314D40033DAE400B399DA0033D7EA0059
:10612000935A0401B394D40093850A0013050A001E
:10613000336B9700EF0010041309050093850A00E4
:1061400013050A00931B0401EF00407E93DB0B0153
:10615000930405009305050013850B00EF00407ABA
:106160001319090113570B013367E900138A04005F
:10617000637EA70033078700138AF4FF63688700F4
:106180006376A700138AE4FF33078700B304A740B0
:1061900093850A0013850400EF00C07D13090500F4
:1061A00093850A0013850400EF00407893040500EE
:1061B0009305050013850B00EF00807413170B0186
:1061C0001357070113190901B367E9001387040086
:1061D00063FEA700B38787001387F4FF63E8870097
:1061E00063F6A7001387E4FFB3878700131A0A0139
:1061F000B384A740336AEA006FF0DFDF63ECD51E9B
:10620000B707010063F4F6041307F00FB335D700A6
:106210009395350033D7B60097A701009387870978
:10622000B387E70003C70700130A00023307B7006C
:10623000330AEA4063160A0213041000E3E096E80A
:1062400033B6CA00134416006FF05FE7B7070001CA
:1062500093050001E3E0F6FC930580016FF09FFBDE
:10626000B35CE600B3964601B3ECDC0033D4E40043
:1062700093DB0C01B397440133D7EA0093850B00FD
:1062800013050400336BF700B3194601EF00806E6D
:106290001309050093850B0013050400139C0C01E2
:1062A000EF00C068135C0C01930405009305050022
:1062B00013050C00EF00C0641319090113570B01FB
:1062C0003367E90013840400637EA7003307970156
:1062D0001384F4FF636897016376A7001384E4FFD7
:1062E00033079701B304A74093850B00138504007F
:1062F000EF0040681309050093850B001385040027
:10630000EF00C062930405009305050013050C001F
:10631000EF00005F93170B011319090193D70701D1
:10632000B367F9001386040063FEA700B3879701E3
:106330001386F4FF63E8970163F6A7001386E4FF72
:10634000B387970113140401B70B01003364C40031
:106350001389FBFF337D240133F92901B384A7405E
:106360009305090013050D00EF008059935C0401AB
:1063700093050900130B050013850C00EF0040582E
:1063800093D90901130C05009385090013850C00AE
:10639000EF000057130905009385090013050D0050
:1063A000EF0000563305850193570B013385A70095
:1063B000637485013309790193570501B387270178
:1063C00063E6F402E392F4BCB70701009387F7FF9A
:1063D0003375F50013150501337BFB0033964A0135
:1063E00033056501130A0000E37AA6CC1304F4FF19
:1063F0006FF09FB9130A0000130400006FF01FCC68
:10640000130101FB2324810423229104232E310351
:10641000232291032326110423202105232C410349
:10642000232A510323286103232671032324810394
:106430002320A103232EB101930C050093890500AD
:106440001304050093840500639E062613090600C5
:10645000138A060097AA0100938ACAE563F4C5145B
:10646000B70701006376F6129307F00F63F4C700D5
:10647000130A8000B3574601B38AFA0003C70A0023
:106480001305000233074701330AE540630C0A0095
:10649000B395490133D7EC0033194601B364B70013
:1064A00033944C01935A090193850A001385040023
:1064B000EF00404C9309050093850A00131B090166
:1064C00013850400EF008046135B0B019305050064
:1064D00013050B00EF00C042939909019357040183
:1064E000B3E7F90063FAA700B387270163E6270142
:1064F00063F4A700B3872701B384A74093850A00FC
:1065000013850400EF0000479309050093850A00F6
:1065100013850400EF008041131404019305050066
:106520009399090113050B0013540401EF00403D3A
:1065300033E48900637AA4003304240163662401F0
:106540006374A400330424013304A440335544018C
:10655000930500008320C1040324810483244104A3
:10656000032901048329C103032A8103832A4103E8
:10657000032B0103832BC102032C8102832C4102D4
:10658000032D0102832DC101130101056780000065
:10659000B7070001130A0001E36EF6EC130A80014D
:1065A0006FF05FED631A06009305000013051000FD
:1065B000EF00C03713090500B7070100637AF90E31
:1065C0009307F00F63F42701130A8000B3574901C2
:1065D000B38AFA0003C70A0013050002B3842941F5
:1065E00033074701330AE540E30E0AEA331949014C
:1065F000B3DAE900B395490133D7EC0093540901AC
:10660000336BB70013850A0093850400EF008036D2
:106610009309050093850400931B090113850A0063
:10662000EF00C03093DB0B019305050013850B00D1
:10663000EF00002D9399090193570B01B3E7F9007F
:1066400033944C0163FAA700B387270163E627015F
:1066500063F4A700B3872701B38AA740938504009A
:1066600013850A00EF0000319309050093850400AB
:1066700013850A00EF00802B9305050013850B009E
:10668000EF00002893150B019399090193D505019B
:10669000B3E5B90063FAA500B385250163E62501DA
:1066A00063F4A500B3852501B384A5406FF09FDF97
:1066B000B7070001130A0001E36AF9F0130A800129
:1066C0006FF0DFF0E3E8D5E8B707010063FCF604FC
:1066D000930BF00F33B5DB001315350033D7A6004D
:1066E00097A70100938707BDB387E70083CB070017
:1066F00093050002B38BAB00338B7541631E0B0215
:1067000063E4360163EACC003384CC40B386D940DD
:1067100033B58C00B384A6401305040093850400B0
:106720006FF05FE3B707000113050001E3E8F6FA35
:10673000130580016FF09FFAB3966601335D760111
:10674000336DDD0033D47901B395690133DC7C010D
:1067500093540D01336CBC001305040093850400B1
:10676000B31A6601EF000021130A050093850400A7
:106770001305040033996C01931C0D01EF00001BFD
:1067800093DC0C01130405009305050013850C0030
:10679000EF000017131A0A0113570C013367EA00C0
:1067A000130A0400637EA7003307A701130AF4FF4E
:1067B0006368A7016376A700130AE4FF3307A70104
:1067C000B309A7409385040013850900EF00801AE0
:1067D000938504001304050013850900EF000015DC
:1067E000930505009304050013850C00EF0040118C
:1067F00093150C011314040193D50501B365B4007E
:106800001387040063FEA500B385A5011387F4FF79
:1068100063E8A50163F6A5001387E4FFB385A5012E
:10682000131A0A01B70C0100336AEA001384FCFF53
:10683000B3778A0033F48A00B384A5401385070038
:10684000930504002326F100135A0A01EF00400BC0
:10685000930905009305040013050A00EF00400AA0
:1068600013DC0A01930D050093050C0013050A00C3
:10687000EF0000098327C100130A050093050C00EF
:1068800013850700EF00C0073305B50113D70901D1
:106890003307A7006374B701330A9A01B7070100F1
:1068A0009387F7FF935507013377F7001317070115
:1068B000B3F7F900B3854501B307F70063E6B40009
:1068C000639EB400637CF90033865741B3B7C700B9
:1068D000B385A541B385F54093070600B307F9409A
:1068E0003339F900B385B440B3852541339475013C
:1068F000B3D767013365F400B3D565016FF09FC569
:10690000130605001305000093F6150063840600C6
:106910003305C50093D5150013161600E39605FE42
:10692000678000006340050663C605061386050000
:10693000930505001305F0FF630C06029306100093
:10694000637AB6006358C0001316160093961600BB
:10695000E36AB6FE1305000063E6C500B385C540D3
:106960003365D50093D6160013561600E39606FE3F
:106970006780000093820000EFF05FFB1385050045
:10698000678002003305A04063D80500B305B0401E
:106990006FF0DFF9B305B04093820000EFF01FF90C
:1069A0003305A040678002009382000063CA05009F
:1069B000634C0500EFF09FF7138505006780020028
:1069C000B305B040E35805FE3305A040EFF01FF6D5
:1069D0003305B0406780020097A70100938747B84E
:1069E000944317A70100130767B61843C8C2637B17
:1069F000E50017A70100130727B608438C4391054C
:106A00006F901FB4411122C406C617A701001307D7
:106A1000E7B42A8408438C439105EF907FB297A78F
:106A200001009387E7B09C436376F40097A70100C9
:106A300023A087B0B24022444101828097A7010081
:106A4000938707B2984394437C43FD177CC3FC4271
:106A500099E3736004308280011122CC26CA2A8413
:106A6000AE844AC84EC652C456C206CEEFB0EFD569
:106A70001C4003290401B7090001B3E59700930AFC
:106A8000C4000CC08144FD19370A00021840638C11
:106A90002A03032609004A85B3654701B376360108
:106AA00093175600758F0329490063C4070001E757
:106AB000F1BFE39DE6FC9317760063D30700D58C06
:106AC000EFC00FC0E1B793C4F4FFF98C04C0EFB07E
:106AD000CFF40840F2406244D2444249B249224ACB
:106AE000924A05618280411106C622C4EFE02FE878
:106AF00017E7FFFF1307475B8146054693054006EE
:106B000017A5010013050590EFD08F8F19C92A84AE
:106B1000EFB0AFCC2A860147814685452285EFD06C
:106B2000CF9AEFB00FA5B2402244014541018280C7
:02000004800278
:100000008A47FEFF8848FEFF9247FEFF8848FEFFB2
:100010008848FEFF8848FEFF8848FEFFAA47FEFF8B
:100020008848FEFF8848FEFFC447FEFFD047FEFF1A
:100030008848FEFFE247FEFFEE47FEFFEE47FEFF69
:10004000EE47FEFFEE47FEFFEE47FEFFEE47FEFFE8
:10005000EE47FEFFEE47FEFFEE47FEFF8848FEFF3D
:100060008848FEFF8848FEFF8848FEFF8848FEFF5C
:100070008848FEFF8848FEFF8848FEFF8848FEFF4C
:100080008848FEFF8848FEFF8848FEFF8848FEFF3C
:100090008848FEFF8848FEFF8848FEFF8848FEFF2C
:1000A0008848FEFF8848FEFF8848FEFF8848FEFF1C
:1000B0008848FEFF8848FEFF8848FEFF8848FEFF0C
:1000C0008848FEFF8848FEFF8848FEFF8848FEFFFC
:1000D0008848FEFF8848FEFF8848FEFF8848FEFFEC
:1000E0008848FEFF8848FEFF8848FEFF8848FEFFDC
:1000F0008848FEFF8848FEFF8848FEFF8848FEFFCC
:100100002248FEFF3848FEFF8848FEFF8848FEFF71
:100110008848FEFF8848FEFF8848FEFF8848FEFFAB
:100120008848FEFF7E48FEFF8848FEFF8848FEFFA5
:100130003046FEFFE846FEFF8848FEFF8848FEFF87
:100140001E47FEFF8848FEFF7647FEFF8848FEFFF9
:100150008848FEFFA447FEFF964BFEFFEA4BFEFFDA
:100160009E4BFEFFEA4BFEFFEA4BFEFFEA4BFEFF13
:10017000EA4BFEFF904AFEFFEA4BFEFFEA4BFEFF12
:10018000AA4AFEFFB64AFEFFEA4BFEFFC84AFEFF40
:10019000D44AFEFFD44AFEFFD44AFEFFD44AFEFFF3
:1001A000D44AFEFFD44AFEFFD44AFEFFD44AFEFFE3
:1001B000D44AFEFFEA4BFEFFEA4BFEFFEA4BFEFF8E
:1001C000EA4BFEFFEA4BFEFFEA4BFEFFEA4BFEFF67
:1001D000EA4BFEFFEA4BFEFFEA4BFEFFEA4BFEFF57
:1001E000EA4BFEFFEA4BFEFFEA4BFEFFEA4BFEFF47
:1001F000EA4BFEFFEA4BFEFFEA4BFEFFEA4BFEFF37
:10020000EA4BFEFFEA4BFEFFEA4BFEFFEA4BFEFF26
:10021000EA4BFEFFEA4BFEFFEA4BFEFFEA4BFEFF16
:10022000EA4BFEFFEA4BFEFFEA4BFEFFEA4BFEFF06
:10023000EA4BFEFFEA4BFEFFEA4BFEFFEA4BFEFFF6
:10024000EA4BFEFFEA4BFEFFEA4BFEFFEA4BFEFFE6
:10025000EA4BFEFFEA4BFEFF084BFEFF364BFEFF6C
:10026000EA4BFEFFEA4BFEFFEA4BFEFFEA4BFEFFC6
:10027000EA4BFEFFEA4BFEFFEA4BFEFF8C4BFEFF14
:10028000EA4BFEFFEA4BFEFFEE48FEFFE849FEFFA9
:10029000EA4BFEFFEA4BFEFF5A4AFEFFEA4BFEFF27
:1002A000804AFEFFEA4BFEFFEA4BFEFFE44BFEFFF7
:1002B000000102020303030304040404040404040D
:1002C00005050505050505050505050505050505DE
:1002D00006060606060606060606060606060606BE
:1002E00006060606060606060606060606060606AE
:1002F000070707070707070707070707070707078E
:10030000070707070707070707070707070707077D
:10031000070707070707070707070707070707076D
:10032000070707070707070707070707070707075D
:10033000080808080808080808080808080808083D
:10034000080808080808080808080808080808082D
:10035000080808080808080808080808080808081D
:10036000080808080808080808080808080808080D
:1003700008080808080808080808080808080808FD
:1003800008080808080808080808080808080808ED
:1003900008080808080808080808080808080808DD
:1003A00008080808080808080808080808080808CD
:1003B000546D725100000000546D7220537663003A
:1003C000286E756C6C2900004572726F7220696E20
:1003D00020787878207461736B73200D0A00000018
:1003E0006D69616F750A00006D69616F75320A0091
:1003F00068756E6772790A0054696D657232000023
:10040000436865636B54696D65720000536574548D
:0C04100078000000536574527800000072
:10041C001000000000000000017A5200017C010174
:10042C001B0D020050000000180000009454FEFF49
:10043C005805000000440E507489039406990B81F2
:10044C0001880292049305950796089709980A9AD1
:10045C000C9B0D036C010AC144C844C944D244D35B
:10046C0044D444D544D644D744D844D944DA44DBA4
:10047C00440E00440B0000004C0000006C00000017
:10048C009859FEFFDC05000000440E30708903957E
:10049C00078101880292049305940696089709989F
:1004AC000A990B9A0C0370020AC144C844C944D27D
:1004BC0044D344D444D544D644D744D844D944DA5C
:1004CC00440E00440B00000050000000BC00000073
:1004DC00245FFEFF0005000000440E507488028962
:1004EC00039305990B81019204940695079608973E
:1004FC0009980A9A0C9B0D0320010AC144C844C9EF
:10050C0044D244D344D444D544D644D744D844D913
:0C051C0044DA44DB440E00440B000000F5
:1005BC00FC8F010009000000FFFF0000FFFF00009E
:0405CC00010000002A
:040000058000004037
:00000001FF
